:020000040800F2
:10000000D81D0020CD000008C13D000835180008AB
:1000100000000000000000000000000000000000E0
:100020000000000000000000000000001D53000858
:100030000000000000000000F140000879610008A5
:10004000DF00000800000000DF000008DF000008FB
:10005000DF000008DF000008DF000008DF00000804
:1000600000000000DF000008890A0008290B0008D2
:10007000DF000008DF000008DF00000800000000CB
:10008000DF0000088562000800000000DF000008B3
:10009000DF000008DF000008DF000008DF000008C4
:1000A000DF00000801530008DF0000089D6200081F
:1000B000256300080348854600F092FB004800478E
:1000C000196E0008D81D00200844F04704488047F6
:1000D00004480047FEE7FEE7FEE7FEE7FEE7FEE72F
:1000E00029620008B500000830B50B460146002023
:1000F0002022012409E00D46D5409D4205D31D462E
:100100009540491B2546954040191546521E002D25
:10011000F1DC30BD70B500242546002801DA012449
:100120004042002901DA01254942FFF7DDFFAC42D8
:1001300000D04042002C00D0494270BDF8B50024E8
:100140002546002904DA0E46012400214042B1412F
:10015000002B04DA1E46002352420125B34100F071
:100160004FFA8C4617461E46AC4203D0002540424B
:100170008D41AC46002C02D0002657429E4161467C
:100180003A46334601B0F0BD10B5202A04DB0846DC
:10019000203AD040002110BD0B46D340D04020244F
:1001A000A21A91400843194610BD03460B439B0712
:1001B00003D009E008C9121F08C0042AFAD203E0DC
:1001C0000B780370401C491C521EF9D27047D2B202
:1001D00001E00270401C491EFBD270470022F6E786
:1001E00010B513460A4604461946FFF7F0FF2046AD
:1001F00010BD0321001D401E037812021A43491E40
:10020000F9D5104670470000F0B50746084658403B
:1002100087B0C00F049048000E46590040084908B6
:10022000BC1A884105D2384631461E4617460B4651
:1002300002465800400810434CD0300D0390400552
:100240005900400D490D0590401A0290402872DA7D
:1002500018030121000B090508430190049800923E
:10026000002805D001995242002088410092019057
:10027000029840210A1A0199009800F0F1F9054608
:100280000C466B4607CB00F0FBF9C0197141039A8D
:100290000E0D0023D71756401A467A40164344D015
:1002A000049A002A2DD0029A012A039A15DC12051D
:1002B000C01A914101263605001C7141D20F059EDE
:1002C000D2070093019202962A46234600F0F8F9DD
:1002D00007B0F0BD38463146FAE71605224A0F4608
:1002E000B218C01AB74101210905001C4F4100187E
:1002F0007F41114618187941E20F10436D1964418E
:1003000013E0E2076D0815436408C2071443039A1B
:1003100001261205C01A91413605001C7141CE0715
:10032000400830434908C01851412A46234600F08E
:10033000BAF9CDE7FFE7049801224000C117121A6D
:1003400000238B4104983146C417381AA141EEE7C7
:1003500030B40124E407634030BC55E730B40124D5
:10036000E407614030BC4FE70000E0FFF0B51FB488
:1003700088B00B990998002448400999C00F49009A
:1003800049080991C0070B990090490049080B9151
:1003900009990898A64608431CD00B990A98084367
:1003A00018D0099801244000420D4800410D0998D9
:1003B00024050003000B204309900B980003000B59
:1003C00020430B9050181C494018002201901446FD
:1003D000104605E0002001460DB0F0BD032801DA0B
:1003E000034600E003239C46C11A0AAE0AE05F0000
:1003F00008ADED5B4F00F75B7D430027AA187C41F9
:10040000491C5B1E6145F2DD410004AB5A522104D8
:10041000120C0A43240C401C0828DFDB01980290D0
:100420000099704601910090059B049A07990698DF
:1004300000F046F9D0E700000DFCFFFFF0B50C46D8
:100440005C4085B0E40FE40703944C000026640888
:1004500059009446490802460296224321D062463A
:100460000A431ED06200570D4A000E032303550DA8
:10047000012402462C492405781B1B0B360B40181F
:1004800023432643614600901C46501AB44103D3CF
:100490000098401C009002E0921800985B410028F0
:1004A00003DA0020014605B0F0BD00200121090556
:1004B0000746864611E064461D46141BB54106D327
:1004C0006546521BB341744607430C43A646CD070D
:1004D00040084908284392185B4105460D43EAD17C
:1004E0001046184313D060461946504071400843E7
:1004F00006D06046101AB34106D20122002306E05E
:1005000000220123DB0702E00122D24353100098AE
:1005100074460105381C6141029C039D0019694124
:1005200000F0C1F8BFE70000FD03000070B54B000C
:100530005B0803430BD04B005C0D0026334665423D
:10054000B341D417AD1AA34102DB0020014670BDB0
:1005500012053018514170BD0EB5C217C10F504081
:10056000CA0740180021054B0293019200910A46E8
:100570000B4600F0A5F803B000BD000033040000F6
:100580000EB505490291002100910A460B460191E2
:1005900000F096F803B000BD330400004A000903E0
:1005A0000123090B1B051943094B10B5520D9A4243
:1005B00001DA002010BD064B34339A4203DC9A1A4C
:1005C000FFF7E2FD10BD03495118884010BD00003F
:1005D000FF030000CDFBFFFF10B5002904DB012461
:1005E000E40740428C412146002B04DB1C460123DA
:1005F000DB075242A341994200D1904210BD000056
:10060000F0B51FB40646002082B005464024019193
:1006100000901BE0019922460F463046FFF7B4FDDB
:10062000049A059B801A994110D310461946224618
:1006300000F016F8361A8F4101972246012000215A
:10064000009F00F00DF838184D4100902046641EC0
:100650000028DFDC019B00982946324607B0F0BD38
:1006600010B5202A04DB0146203A9140002010BD3D
:10067000914020239C1A0346E3401943904010BD4B
:1006800010B5202A06DBCB170846203A1041C117C7
:100690000B4306E00B461341D0402024A21A9140A0
:1006A0000843194610BD10B5002B08DA0024401C81
:1006B000614192185B411A4301D14008400010BDCE
:1006C000F0B51FB482B005460C0003D0084605F013
:1006D000CBFF02E005F0C8FF203002460090214623
:1006E0002846FFF7BDFF049B059A04460F461843B2
:1006F0001143084314D0184610431BD000984021E2
:100700000A1A18460599FFF73FFD05460E46009A5E
:1007100005990498FFF7A4FF084305D0012004E0E1
:100720002046394607B0F0BD0020C11705430E43EF
:100730002C43374300990E986305401A7905E40A63
:1007400000220C43FD0A0A3002D500200146E9E7E9
:100750000105101969410C9C0D9D00196941FFF7B5
:10076000A2FFDFE7F8B50546480040080C462843DD
:1007700004D06000184A400D904201DD2846F8BDC3
:1007800015493539884210DC88420BDB290D2003DE
:1007900008432903014305D0E00F1049C007411861
:1007A0000020F8BD00200146F8BD161A4020821B2B
:1007B00028462146FFF754FF074600912846214668
:1007C0003246FFF7E1FC3A46009BFFF76CFF3246EA
:1007D000FFF746FFF8BD0000330400000000F03FC3
:1007E000064C0125064E05E0E36807CC2B430C3C84
:1007F00098471034B442F7D3FFF760FC64790008DF
:100800008479000870B58C180578401C6B075B0F65
:1008100001D10378401C2A1106D10278401C03E064
:1008200006780E70401C491C5B1EF9D12B0705D4BD
:100830000023521E0DD40B70491CFAE70378401CAC
:10084000CB1A921C03E01D780D70491C5B1C521ED4
:10085000F9D5A142D8D3002070BD0000F0B51C4AE4
:1008600090684007C00F31D1106C1B4D81B2194800
:100870001A4B04690120E607002E0AD09982184C11
:10088000184B2846A14201D2012100E00021196045
:1008900012E0A54306D0144DA54306D0134DA54341
:1008A00006D009E01983124806E01984114803E0D4
:1008B00059841149498BD9834103490B916291684D
:1008C0000E4B1940091D9160024908610020F0BDDE
:1008D000002401400000002000010020C01300207F
:1008E00098080000BC000020000001400000024405
:1008F000000001C0000002C4A0F7FF1FE8FFFF7F57
:10090000F0B51C4C85B025691B4E6D1C2561376800
:10091000B668029600976E467580019031817281AB
:100920000393206A01011548091800200A5CFF2A78
:1009300004D01022304600F03FF906E0401C102899
:10094000F4D31022304605F055FE206AE061401CC9
:1009500020620001012109031030884201D90020E2
:100960002062E0680649401CE0604867002005B04E
:10097000F0BD0000980000201078000800D00008AA
:1009800040130020002911D0826852188260436809
:10099000934200DCD21A00238361C368934201D1E1
:1009A0000123436182600269521802610846704760
:1009B000FCB51D4801901E4D0020E860EA692B69D6
:1009C00094466A6900922A6AAD69184C0146AE469F
:1009D00013E0665B174FBE420ED12E197588401C7E
:1009E0009D4204D9726800922B468C464A1C019E97
:1009F000B54201D28E460195491C01260D013603F0
:100A0000B542E6D30A490B616346CB61009B4B615B
:100A10000A62C860734612018B61334610329A42F3
:100A200001D900220A62FCBDFFC99A3B00D0000830
:100A300098000020AA55000010B50421054800F0D8
:100A4000DCF8054800218161C1610161C16001627A
:100A5000084610BD00D000089800002030B50023E3
:100A6000040AE409CD09E401ED01AC4203D04004DD
:100A7000000C504001E04004000C49065B1C090ECC
:100A8000DBB2082BECD330BD70B5234CE06A401CC0
:100A9000E062224E30688006C00F11D02068216BC2
:100AA00040182060216B20465830054600F058F869
:100AB00020207060A86900280AD00020206360729E
:100AC00030688005C00F02D001204002706070BD08
:100AD000284600F07FF912494A78B3585B085B005A
:100AE000B350EB682A684D78D2180C4B0C33EA509F
:100AF0000A4A4B78121D9D582D0C2D0405439D501C
:100B00004978725801231A4372502063054881685E
:100B1000802211438160D3E7E00200200000024000
:100B200025780008003801400B48C16A491CC162A1
:100B30000A490A689204D20F05D0012252034A6082
:100B400000220263427208688003C00F02D00120B5
:100B50004004486070470000740300200000024019
:100B600010B5002910D0C26843685218934200DCC7
:100B7000D21A00234361C2608468944204D10122E6
:100B800082618360C360C361084610BDFF210922F2
:100B90000131D206002801D09162704791617047FF
:100BA00001218902034A002801D0916270479161B6
:100BB0007047000000040048F0B585B016460D46A9
:100BC000074600F077FA012002900020009001957E
:100BD00003A9684600F0D6F90024760807E0600013
:100BE0003A5A41190023012000F026FA641CA6425B
:100BF000F5D800F017FA05B0F0BD7FB50D460446F4
:100C000000F058FA00206A4631C203A9684600F095
:100C1000B9F900F007FA04B070BD000006490020E1
:100C2000C86106480169042211430161016940223B
:100C30001143016170470000B819002000200240F4
:100C4000064A0021D16106490A6902231A430A6152
:100C5000486108694022104308617047B8190020B4
:100C60000020024010B5054B0022DA61044A1369E6
:100C7000012423431361018010BD0000B819002036
:100C80000020024010B50B4A0020D168CB060A496B
:100C900004D5C86902231843C8611020D3685B07D4
:100CA00005D5CB6901242343CB6104210843D060DF
:100CB00010BD000000200240B819002070B50546A4
:100CC00000F00AFA0646104C0AE0681C08D0002D15
:100CD00004D000F001FA801BA84201D9032070BDA6
:100CE000E068C007F1D1E068800601D52020E0600F
:100CF000E068C00602D4E068400703D5FFF7C2FFF2
:100D0000012070BD002070BD002002400A07120FB4
:100D100001219140014201D001207047002070471D
:100D20000A07120F01219140014201D001207047B2
:100D300000207047F8B50A05120E254B5200D21854
:100D400009239B01D31800930523DB01D618012347
:100D500005469B020C07D7180020240F2B0005F036
:100D60009AFC09060A0E12191D21282F2E00FF29B0
:100D700028D800981BE0FF2924D8009808E0FF2914
:100D800020D8B08A18E080291CD20F2080011018CA
:100D9000808E11E0802915D2B88A0DE0402911D249
:100DA000B08E09E040290DD20B2080010EE0808A30
:100DB00002E0802906D2B88E2146FFF7B1FFF8BDC8
:100DC000802901D30020F8BD0920C0011018EEE7EA
:100DD000C00D0020C1688268914201DA501A704744
:100DE000914202DC4269002A02D04068401A7047F2
:100DF00080690028FBD000207047C268816891425A
:100E000001DA501A7047914202DC8269002A02D04E
:100E10004068401A704740690028FBD000207047A6
:100E2000064901228969120308180101914201D380
:100E3000FF3801380249000140187047980000202F
:100E400000D0000800B5102000F094FD00BD0000A7
:100E5000014840687047000018000020F0B5334B8F
:100E60004A00D2180923DB01D4180B230546DB0105
:100E70000020D318892D25D00EDC2C4F2C4B4E0092
:100E8000F619F618803D2B0005F005FC091F1F150B
:100E90002125292E333A15008D2D3FD00CDC8A2DCB
:100EA00033D08B2D35D08C2D05D140293ADA0B204B
:100EB00080011018808EF0BD992D03D0A12D01D096
:100EC000FE2DF8D180292DDA2EE00846F0BD10293C
:100ED00028DAB08AF0BD102924DAB08EF0BD1029CE
:100EE00020DA0520C00108E008291BDA0F20800164
:100EF000DFE7082916DA012080021018808AF0BD89
:100F000080290FDA3420205EF0BD80290ADAA08A19
:100F1000F0BD402906DA0D208001CAE7402901DA38
:100F2000A08EF0BD0020F0BD988EF0BDC00D002059
:100F30004002000010B507488168074B9A69846831
:100F4000A14201D081689A69044842431014081AEA
:100F500010BD00001800002000E000E05505000072
:100F600031B500F0B9F8009C0546601C00D0641C47
:100F700000F0B2F8401BA042FAD338BD10B5FFF71D
:100F8000EFFF10BDF8B5054623480F46017E012648
:100F900001290BD0012101762868204C012807D0B7
:100FA0002046FFF78BFE002813D030E00220F8BD6A
:100FB0002046FFF783FE002829D1FFF72FFE2046A9
:100FC000FFF77CFE06461648016904229143016141
:100FD0001DE00020C04338606C6812E02046FFF737
:100FE0002FFE0E48FFF76AFE06460D4802690221F1
:100FF0008A430261002E01D03C6008E0012080029B
:101000002418A868810268680818A042E6D8024837
:10101000002101763046F8BDB819002050C3000009
:101020000020024003480169802211430161002031
:101030007047000000200240F0B51FB407461A4870
:101040000024017E15461E46012907D001210176A4
:101050001648FFF733FE002803D020E0022005B039
:10106000F0BD012F02D0022F00D004272201284614
:101070003146FFF789F881B2019862001018FFF736
:10108000F1FD0A48FFF71AFE09490A6952085200A1
:101090000A61002803D1641CE4B2BC42E6D30249D1
:1010A00000220A76DBE70000B819002050C30000D8
:1010B0000020024005480169090605D50449416040
:1010C0000449416000207047012070470020024021
:1010D00023016745AB89EFCD0148006870470000E8
:1010E000DC01002002480168491C016070470000D3
:1010F000DC01002010B50648016810221143016090
:10110000002000F007F800F017F8002010BD0000E4
:101110000020024010B5044600F03EF97D21C900D0
:10112000FEF7E2FF00F06AFB00222146501E00F0AD
:1011300025F8002010BD000008B50F488169012284
:1011400011438161816911400091C26901040A4320
:10115000C261C0690022084000901146501F00F093
:101160000DF800221146901E00F008F800221146EA
:10117000501E00F003F808BD0010024010B502F048
:101180004DFE10BDF8B505460068354CC00352D57C
:10119000E0690026C00007D4E16920040143E16151
:1011A000E1690140012600912E480168C90510D46B
:1011B0000168821511430160FFF78EFF074604E0C6
:1011C000FFF78AFFC01B642824D826480068C005A2
:1011D000F6D5206A03273F02384020D0696839409D
:1011E00081421CD0206A226AB843012109040A43C3
:1011F0002262226A8A4322622062C0070FD0FFF770
:101200006BFF009008E0FFF767FF0099411A16484E
:10121000814201D90320F8BD206A8007F3D5206AF6
:101220006968B84308432062002E04D0E1690120B8
:1012300000078143E1612878C00705D0206BA968C9
:1012400080088000084320632878800605D5206B3D
:1012500010218843E968084320630020F8BD00009E
:10126000001002400070004088130000F8B50546E9
:1012700044480E460068C007C00FB0420AD2414839
:10128000016849084900314301600068C007C00F88
:10129000B0425CD128783C4C800705D56068F021CD
:1012A0008843A968084360602878C0073FD0686811
:1012B000012813D02168022813D08907002946DAB3
:1012C00061688908890001436160FFF705FF69686B
:1012D000074601290DD0022917D024E0216889038F
:1012E000ECE78901EAE7FFF7F7FEC11B27488142D7
:1012F00017D860680007800F0128F4D117E0FFF7C6
:10130000EBFEC11B214881420BD860680007800FAB
:101310000228F4D10BE0FFF7DFFEC11B1B4881421E
:1013200001D90320F8BD60680007800FF3D115488C
:101330000168C907C90FB1420BD9016849084900C2
:10134000314301600068C007C00FB04201D00120E6
:10135000F8BD2878400706D5606807210902884350
:10136000E9680843606000F01DF86168084A0906F2
:10137000090F515CC840074908600020FFF7CAFE0A
:101380000020F8BD00200240001002408813000039
:101390004C790008D801002001480068704700001F
:1013A000D801002010B512A30FCB88B06C460FC433
:1013B00013A30FCB0FC416494A680C2013460340F1
:1013C0001448042B0FD0082B0DD193021B0F6C4631
:1013D000E45CC96A04AB0907090F595CD20304D560
:1013E000FEF782FE604308B010BD0B486043FAE789
:1013F00002030405060708090A0B0C0D0E0F101056
:101400000102030405060708090A0B0C0D0E0F1054
:101410000010024000127A0000093D00FEB50446AB
:101420000078D04DC00747D068680007800F0128BA
:1014300007D068680007800F022809D16868C003D8
:1014400006D52868800337D5606800287ED033E051
:10145000012062680004012A11D08100002A01D015
:10146000052A10D02A6882432A60286888432860A9
:101470006068002814D0FFF72FFE06460CE02968AC
:1014800001432960F4E72A680A432A60F7E7FFF777
:1014900023FE801B64286FD828688003F7D50BE0F3
:1014A000FFF71AFE064604E0FFF716FE801B6428CD
:1014B000F1D828688003F7D4207801268007002817
:1014C0003BDA68680007800F07D068680007800F64
:1014D000022809D16868C00306D42868800715D59A
:1014E000E068012832D111E0E0680028286815D0B2
:1014F00030432860FFF7F0FD074604E0FFF7ECFDFE
:10150000C01B0228C7D828688007F7D52868F821AB
:1015100088432169C900084328600EE04008400064
:101520002860FFF7D9FD074604E0FFF7D5FDC01B93
:101530000228B0D828688007F7D42078000724D57F
:10154000E0690028686A10D0304300E008E1686272
:10155000FFF7C2FD074604E0FFF7BEFDC01B0228EF
:1015600099D8686A8007F7D50FE0400840006862A4
:10157000FFF7B2FD074605E09DE0FFF7ADFDC01B9C
:10158000022888D8686A8007F7D4207804274007A3
:10159000002860DA00200190E869C00008D4E969F9
:1015A000B8060143E961E969014001200091019019
:1015B0006D480168C90511D40168821511430160A5
:1015C000FFF78AFD009005E0FFF786FD0099401ABD
:1015D000642870D864480068C005F5D5A068012863
:1015E0000AD0002801D0052810D0286A4008400001
:1015F0002862286AB84301E0286A30432862A0685C
:10160000002812D0FFF768FD00900AE0286A3843EE
:101610002862F1E7FFF760FD0099411A53488142C3
:1016200049D8286A8007F5D50DE0FFF755FD0090F1
:1016300006E0FFF751FD0099411A4C4881423AD823
:10164000286A8007F5D40198002804D0E9690120B0
:1016500000078143E9612078C00635D5606901281B
:101660000CD0401D686B23D038436863686B40081A
:1016700040006863FFF730FD064622E0686B3843A0
:101680006863686B30436863FFF726FD064604E035
:10169000FFF722FD801B02285BD8686B8007F7D517
:1016A000686BF8218843A169C900084368630BE0AF
:1016B000B8436863F4E74CE0FFF70EFD801B022897
:1016C00047D8686B8007F7D4206A002846D069683D
:1016D0000907890F022943D0012636060228286807
:1016E00005D0B0432860FFF7F7FC044633E0B04371
:1016F0002860FFF7F1FC074604E0FFF7EDFCC01B94
:10170000022826D828688001F7D4E86AE16A00092F
:1017100000010843E862616AA06A084369683D22E3
:101720001204914308436860286830432860FFF73B
:10173000D3FC044604E0FFF7CFFC001B022808D8C6
:1017400028688001F7D509E0FFF7C6FC001B0228D6
:1017500001D90320FEBD28688001F5D40020FEBD1C
:101760000120FEBD00100240007000408813000000
:10177000042204490428086902D090430861704794
:101780001043FBE700E000E01548016864310160A8
:1017900014480168491C016013480168491C016034
:1017A0001249134AC868401CC860904216DB0020EA
:1017B000C8601048816D491C8165016D491C016537
:1017C000416D491C41650C48018B002906D0491E1A
:1017D00089B20183782901D97821018370470000FB
:1017E000200000201C00002068000020C80000200D
:1017F000102700004013002074150020094910B57F
:10180000401E884201D9012010BD074C60610321B0
:10181000081F02F003FB0020A061072020610020C8
:1018200010BD0000FFFFFF0000E000E010B5FFF773
:10183000ABFF10BDFEE7000010B500200F4A0146C7
:1018400050604B009B18491C1881FF29F9DD0021CD
:1018500005230B4ADB014C00A418E418491CA082A4
:101860001029F8DB00210923DB014C00A418E4183F
:10187000491CA086FF29F8DD002010BD380B002090
:10188000C00D002010B5402802DB0020C04310BD71
:1018900010221143C200094B4000D218C01858242E
:1018A0000D23A1529B010021C3189986E300C018A3
:1018B0008186034800685065084610BDC00D0020B1
:1018C000DC01002070B504461E463830049D05F04A
:1018D00097FA20462A463146583005F091FA002002
:1018E00070BD000070B5104D064601462846FEF753
:1018F00011FC0E4C6061FFF74FFD2946FEF7F4FB2B
:10190000E0600B48314600680546FEF7EDFB2061BC
:101910002A46002307480F21FEF710FC208060694B
:101920006430A060002070BD40420F00180000200D
:10193000D80100200000404230B5002372B61022CA
:101940000921C9068A628A61441E0122A240084C0C
:10195000002809D025682D0600D4134320258D6268
:1019600052088D61401EF5D162B6184630BD0000A8
:1019700010000048F8B572B610220921C9068A6223
:101980008A61C217520F1018C71000200B4E00902A
:101990000FE000228024082335686D0600D422431E
:1019A00020258D6264088D615B1EF5D16B461A544B
:1019B000401CB842EDDB62B60098F8BD100000484C
:1019C000034610B50020024602E09C5C6040521CB9
:1019D0008A42FADB10BD0000F8B508460D460978CA
:1019E000552901D0252903D0012A01DD451C521EAD
:1019F000344C602661792B787143334E8919334E0C
:101A0000252B30D0B3685B1CB360CB695B1CCB610A
:101A1000A17800290FD0E17800290FD001292C49A5
:101A200013D007231B02C9180A7501462948FEF77F
:101A3000BCFB0020E0700020C043F8BD2549264BC8
:101A400055390A750146224807E037235B01C9185A
:101A50000A750146204B1E482033C018FEF7A5FB2F
:101A6000E078401CE6E76F79802F06DDF068401CC7
:101A7000F060086A401C0862DDE73B4608339A4282
:101A800008D2086A401C0862F068401CF06002201E
:101A9000C043F8BDB91DFFF793FFE9198979814269
:101AA0000DD03069401C30616179602041430648A7
:101AB0000818416A491C41620320C043F8BD002058
:101AC000F8BD00004C00002028060020F403002090
:101AD000C00D0020D5140020D5060000F8B50E4634
:101AE00005462527079C089906982F706A70AE70E6
:101AF000EB7028712746002008372E19372B1AD093
:101B000009DC1A46303A130004F0C5FD0726151506
:101B1000262626172600612B0DD006DC382B0AD08E
:101B2000412B08D0422B17D105E0622B03D0632B49
:101B300001D0642B10D16C7102E06C71002C03D0C9
:101B40002246A81DFEF731FBA11D2846FFF738FFEE
:101B5000B0710D20F0713846F8BD0000F1B584B0C9
:101B6000FFF7BAFA0546FFF7E5F9604C0646E0795B
:101B7000002806D0207A002803D0E068301A3228E6
:101B800005D8E0687D21301AC90088427ED9207AC4
:101B9000574B00281DD0617960225143554A0120DE
:101BA0005050642058646079401CC0B26071E17A82
:101BB000884208D9A06AA662301AE062A079401C67
:101BC000A071012060714C48008A4C4F002830D031
:101BD00038E0606A401C606249484168491C4160C5
:101BE000617960200A4642434248944610180269CF
:101BF000521C02614269521C4261E779002F02D1F6
:101C0000876A7F1C87628769BA4200D98261394836
:101C1000032AC8D900226746C251C82098643948AF
:101C200042544800384941180F2080010818828624
:101C3000B9E7FFF707F9354980B28882C1B2F98266
:101C4000000A38832F49B87D10314870387E88707B
:101C500062792F488B5C0370891849784170602144
:101C600013464B4323490027C9588170C77005713B
:101C70002B0A43712B0C83712B0EC371E6606E46E9
:101C80003378A6799B089B00B60700E028E0B60FE2
:101C900033436E463370002925D0EF210B4033705B
:101CA0000290082117480093019141230021203020
:101CB000FFF714FF134902462031049803F0E0FFB8
:101CC0006179602041430B4808184168491C416014
:101CD000C268E1688A1A4263C1606563E77127726E
:101CE000002005B0F0BD10210B43D8E74C000020C8
:101CF000401300202806002074150020C011002089
:101D0000F403002008050020C00D00200010002072
:101D100028090020F7B5087886B00C46552801D070
:101D2000252802D0012A00DD4C1C4C4D60796979D0
:101D30006022049151434A4A2B4689188A682F46EB
:101D4000521C8A60464A803A03921B6BFF68E67811
:101D5000DF1B2B46A2789B69303E0093330004F0D2
:101D60009AFC13420B1742424229424242424242EB
:101D7000424242422C4542003A49A3798B5422798F
:101D8000A11D32230092029101900021049A22E0C9
:101D90006F610098874200DDAF613248A3798354B8
:101DA0000020CF624861086BB84200D20F63012067
:101DB000287218E00120E87115E02A49A2790A701A
:101DC00010310978A1712279A11D00920291019030
:101DD0004223297900220398FFF780FE02460399E7
:101DE000069803F04DFF002009B0F0BD6F61009828
:101DF000874200DDAF611B49A079885451001A4A1F
:101E000089180F229201891888861848008A0028AC
:101E100009D11748C18E008F00020818154980B2F9
:101E2000888602F037FD6A7960214A430C49002018
:101E3000561870616869F062316B814200D230637C
:101E40002046677A0A30FEF7D4F9617B0002000A67
:101E500009060843B90071188863A8E74C00002000
:101E60002806002008050020C00D00207415002061
:101E70008011002000100020F7B516460D46FFF730
:101E800059F81A4C206329780020552903D1012ED6
:101E900001DD6D1C761E217800290FD00127E77126
:101EA000324629460098FFF797FD002805D1277292
:101EB000324629460098FFF72DFFFEBD61780029C4
:101EC000FBD00B4C3246A06B2946401CA063009807
:101ED00000F012F80028F0D106483246406C206528
:101EE0002946009800F050F8FEBD00004C0000208C
:101EF0002806002040130020F0B508460C4609785B
:101F0000552901D0252903D0012A01DD441C521E88
:101F1000217800231A4EDB431A4D252906D0A868E4
:101F2000401CA860306C401C306409E0144967799B
:101F3000896C491C802F05DDE868401CE860B164AD
:101F40001846F0BD3B4608339A4206D2B164E868B1
:101F5000401CE8600220C043F0BDB91DFFF730FD12
:101F6000E1198979814208D02869401C2861F06C08
:101F7000401CF0640320C043F0BD0020F0BD000011
:101F800028060020F4030020F7B5087884B00C463A
:101F9000552802D1012A00DD4C1C57480168491C14
:101FA000016066796278554855490390534D087928
:101FB0008035824208D0FF2A06D0686C401C6864D5
:101FC0000020C04307B0F0BD824201D0FF2A7DD17E
:101FD0000A6B00920A6101224A72484AE778A03AE5
:101FE000372F73D007DC303F3B0004F054FB0682F0
:101FF000138282822482612F7BD004DC382F78D038
:10200000412F76D120E0622F73D0632F71D0642FDF
:102010006FD163E0A3791370384A903A1278A271B5
:10202000009A0A612279A11D322300920291019641
:102030000022014644E000202179362300910190DE
:102040000246029001213BE0A0791070E37AA27A67
:102050001B022B49D218CA6102F01CFC2848877A5F
:10206000FEF7F0FE254990390870A071B80067723C
:102070004019018FA172018F090AE172816B090C6D
:102080002173806B1E49000E60731D48807A401CCE
:10209000C0B288720A2801D300208872207969466C
:1020A0000870C00603D57D20164980018864217917
:1020B000A01D02901248019600914223017900224E
:1020C0000398FFF70BFDE96B491C00E011E0E963A1
:1020D00002460399049803F0D3FD0AE0E279A0795F
:1020E00012028018227A637A12041B06D218801812
:1020F000C861002066E70000F4030020A805002066
:102100004C00002040130020034610B5002002467A
:1021100002E09C5C6040521C8A42FADB10BD30B584
:102120000D46084609781446252901D0012030BD06
:10213000062C01D2032030BD611EFFF7E5FF2919EF
:102140002039C97F814201D0042030BD002030BD3C
:1021500070B51E4605465523049C05982B70697082
:10216000AA70EE7001462C712246681DFEF71DF81C
:10217000611D2846FFF7C8FF29194871A01D052ECB
:1021800002DA002E00D1002070BD0000FEB5154619
:102190000E460746FFF7C3FF040014D068460472DA
:1021A0000420009002A90B4801910278401E01789A
:1021B000EE230948FFF7CCFF02460749384603F0F3
:1021C0005FFD2046FEBD2A463146384600F006F83F
:1021D000FEBD000085000020B8090020F7B5FE4ACA
:1021E00086B04F7850689060501C05780B792E09A6
:1021F0008D7836012D072D0F2E430670F74802907B
:1022000010780C460490874201D0FF2F75D12146EB
:10221000E5780931F2488C46332D70D028DCF1493D
:10222000182D0A686AD012DC072D20D008DC002D9A
:1022300063D0012D3ED0032D41D0052D7ED15EE02F
:10224000112D7CD0162D7BD0172DF7D14AE2232DEE
:10225000EED006DC192D74D0212D73D0222DEDD1B6
:1022600098E1242DE4D0312D49D0322DE6D1C2E0C1
:10227000582D68D012DC542D66D008DC342D71D076
:102280004F2D70D0502D6FD0532DD7D179E2552DD1
:102290006BD0562D6AD0572DD0D16FE229466339C5
:1022A00004200B0004F0F7F909F0EFEE151B4A10BB
:1022B0004A134A00641D0093019401235CE2CA4959
:1022C0001820BCE23946D2E2C8490C20B7E2C8491E
:1022D000B5E2C74910395020B1E22B464CE2E17912
:1022E0000020BE4A03E023185B7A1354401C884246
:1022F000F9DBBA4804F024F9AAE082E2FBE1A27912
:10230000617912028918E27989B2882B2FD0892B42
:1023100031D08A2B33D0832B36D0842B39D0852BE8
:102320003CD0862B3FD0872B42D08B2B45D08C2B9B
:1023300048D0FE2B1FD0A92B49D006E0A2E2A9E18C
:10234000B8E1F8E1D2E071E232E2B32B43D0B42B32
:1023500044D0992B46D0A12B49D0A0481038401822
:102360000092BAE147E001E2FCE14BE254E24900AD
:102370000918A04834E0490009189F4830E0490096
:1023800009189C4820382BE0490009189520800046
:1023900026E0490009189D20800021E04900091825
:1023A000A52080001CE049000918FD20800017E0EE
:1023B000490009188F48A03812E049000918DD20AB
:1023C00080000DE049000918BD20800008E04900A8
:1023D00009188A4804E04900894801E08948490011
:1023E0000818BDE7884849000818001DB8E74800EC
:1023F0000121C906B3E7A279617912028918E2794D
:1024000089B2882B27D0892B29D08A2B2BD0832BDC
:102410002ED0842B31D0852B37D0862B3AD0872BEA
:102420003DD08B2B40D08C2B43D0FE2B47D0A92BFB
:1024300049D0B32B4BD0B42B4CD0992B4DD0A12BE2
:102440004FD066481038401800226146FDF7ADFEB7
:102450000020009029E14900091866483FE0490042
:10246000091865483BE0490009186248203836E001
:10247000490009189520800031E0490009189D2085
:1024800080002CE0EAE1DDE1D8E149000918A5204F
:10249000800024E049000918FD2080001FE0490069
:1024A00009185448A0381AE049000918DD208000B6
:1024B00003E049000918BD2080000818C4E749005E
:1024C00009184D48F9E7490009184C48F5E7490053
:1024D0004B48F2E749004B4801E04B4849000818D7
:1024E000B3E748000121C9064018AEE7A279617937
:1024F000120289180922920189B2002B0FD0012BF8
:1025000013D0022B1CD0032B20D0042B26D0052B5C
:102510002AD0062B28D0082B34D000202AE00B0923
:102520005B00181833E0012024E00B095B00181849
:1025300011E00A07120F012191400840F3D119E080
:102540000A09520010180522D20120E00A0952009F
:1025500010180F2292018018808EEAE70A095200B3
:1025600010180122920212E0C90008184030007EC3
:102570004006C00F69460873012003A92123019179
:102580000090F9E00A09520010180922D2018018BF
:10259000808ACEE7A27961791202891889B2002B6C
:1025A00034D0012B3BD0022B42D0032B49D0042B3B
:1025B00050D04022052B55D0062B53D0072B5CD092
:1025C00000206946087300200090034803A9401CBE
:1025D00001910278222375E684000020B8090020CA
:1025E000C00D0020380B002076770008ACF7FF1FE5
:1025F000107C0008B4040000B4050000B40600001C
:1026000028060020B4170020400D00200B07090900
:10261000490009181B0F9520E279800035E00B076F
:102620000909490009181B0F9D20E27980002CE060
:102630000B070909490009181B0FA520E279800042
:1026400023E00B070909490009181B0FFD20E27957
:1026500080001AE00B0709091B0F49000918E279ED
:102660008E4812E0C90008184030018B9143E2798E
:10267000D207520E11430183A5E70B070909490050
:1026800009188648E2791B0F80300818194603F0B4
:102690001BFB98E7002B05D0012B00D0D8E603F0F8
:1026A000F1FCD5E603F026FDD2E601907C48E37804
:1026B000027807E6A179607909024018E179794A40
:1026C00080B2002B0BD0784C012B03D0774B9B8A28
:1026D000002B04D04000001900910190FDE540005E
:1026E0008018F9E7002A01D000200860002000903F
:1026F0001723019040E0002A01D000200860A17952
:1027000060790902401885B2E2790020684903E047
:102710002618767A0E54401C9042F9DB644928460C
:1027200003F01AFF00200934009001905C480394E4
:1027300002781823C6E5A1796079090240185B493F
:10274000C882888A00280BD000208882574803F06E
:102750005BFA002000900190514819230278B1E5FE
:102760000120F2E751480383002002E04F49002096
:10277000088300900190E3783246A3E54B4920207E
:102780005DE0A1796079090240184A4980B20A18CF
:10279000E179121D782801D3002105E00B18782B70
:1027A00002D97821081A81B2C8B20192009094E54A
:1027B000A1796079090240183E4980B20B18E2798C
:1027C0001B1D782801D3002205E01118782902D9B1
:1027D0007821081A82B261461846FDF7E6FC00200F
:1027E000009001902E48E378027839460298FFF76E
:1027F000AFFC02460299069803F042FA2D4803F016
:10280000CBFE3CE02B4803F0C7FE00200090019077
:1028100023485523027855E5244803F0F5F90020B4
:10282000009001901E48562302784BE503210902CF
:102830002148FDF7D3FC002000904EE71F4901918D
:1028400000904AE5A179607909024018E17980B2E7
:102850000D01FEF7E5FAE9B2009126E7FEF7ECF884
:102860000020009001900E48652302782AE5029826
:10287000FFF76EFC02460299069803F001FA002069
:1028800009B0F0BD02206946087303A90120019137
:10289000EE23324600900499E9E70000140400009A
:1028A000850000200080000800A0000874150020AA
:1028B000B8090020400D002028060020B413002095
:1028C00070B5FEF775F8164800F05CFD154C164D16
:1028D0006069A8651248816869658188491C8180A2
:1028E0008088E8640E4803F08FF9206828676068E4
:1028F0006867A068A86701220C4B1146A86DFDF718
:10290000FFFF28468030E1680160A1694160E1690C
:1029100081602169C160216A0161002070BD0000F1
:10292000741500209800002040130020393000006A
:1029300070B50D46881EC1B20122354802F04CF830
:10294000334C344A6119D08020398B7F2546C6B27A
:10295000943DB3420BD0C97F000A814207D0E86C96
:10296000FF21401CE8642C48F53181644DE0284E7D
:102970003078AA2849D150789278717800011043B4
:10298000814242D100F0EAFCFEF762FA2862FEF7CB
:102990005FFAA8620020E863F178304634380029F5
:1029A00004D0012907D0022911D01BE0A17A81723D
:1029B000E17AC17216E0627A217A12028918A27A4B
:1029C000E37A12041B06D2188918E9660AE0627AD3
:1029D000217A12028918A27AE37A12041B06D2180D
:1029E000891829670A214156C07A000208180B4944
:1029F0004042C88061792079090241180848C182A3
:102A0000E279A179120289180183002070BD0000CB
:102A100048180020F000002040130020C0140020BF
:102A20000012002070B52C4855212C4C01706178A3
:102A3000A27809011143417003218170C178264DAC
:102A4000491C8907890FC1702549CA8E0271CA8E37
:102A5000120A42710A8F8271098F090AC171C07806
:102A6000002806D029461039012807D0022809D0AD
:102A70000CE0E078A8722079E87207E016489038F8
:102A8000806A02E014489038C06A88610C210122F3
:102A9000114801F0A1FFE0800F4A2873010A517329
:102AA000104914468884743CE068401CE060FEF7DE
:102AB000CFF96169401A6063FEF7CAF960610A489C
:102AC0000E21826A044890470120A060FEF7C0F9F9
:102AD0006062002070BD000028180020F000002077
:102AE00000120020C01400202C780008F8B50D4614
:102AF0003A4E881EC1B20122304601F06DFF3446C5
:102B0000374A6119D08020398B7F2546C7B2943D62
:102B1000BB420BD0C97F000A814207D0E86CFF217D
:102B2000401CE8642F48F531816448E0307855282E
:102B300045D15078927871780001104381423ED19E
:102B400000F00CFCFEF784F92862FEF781F9A86218
:102B50000020E863F078002804D0012809D002287A
:102B600013D01DE01D48A17A34388172E17AC17218
:102B700016E0617A207A09024018A17AE27A090403
:102B8000120689184018E8660AE0617A207A09027C
:102B90004018A17AE27A09041206891840182867B9
:102BA00061792079090241180F48C182E279A1793F
:102BB000120289180183012000F01AF80BE00B487B
:102BC000416BFA2088470220A860FEF741F968624D
:102BD000FEF73EF9E8610020F8BD0000481800202B
:102BE000F000002040130020001200202C78000884
:102BF00070B52848AA21284C01706178A278090193
:102C00001143417003218170C178224D491C89070D
:102C1000890FC1702149CA8E0271CA8E120A42718F
:102C20000A8F8271098F090AC171C078002806D005
:102C300029461039012807D0022809D00CE0E07895
:102C4000A8722079E87207E012489038806A02E0A2
:102C500010489038C06A88610C2101220D4801F0AB
:102C6000BBFEE08028730B49000A48730C480E2114
:102C7000826A08489047074C0120743CA060FEF728
:102C8000E7F86062E068401CE060FEF7E1F8606130
:102C9000002070BD28180020F00000200012002045
:102CA0002C78000870B5304E706880472F49314C41
:102CB00088862F49097800290DD0FEF7C9F8616987
:102CC000401A7D21090188424BD96068002848D10B
:102CD00000F0CAF845E0254D4035002804D0012811
:102CE00006D0032819D025E0A88A401CA8820FE04E
:102CF000FEF7AEF8E169401A1F4988421AD9FEF77B
:102D0000A7F8E061606D401C6065E88A401CE882BD
:102D1000306B804700F0A8F80CE0FEF799F8E16905
:102D2000401A0A2806D9A06D401CA065288B401CBB
:102D30002883EDE7FEF78CF8216A104D401A7D21BB
:102D40004901884201D9C810A864FEF781F8216AB8
:102D5000401A0B49884204D90A48A8640A4900204D
:102D6000C882002070BD00002C780008801400206C
:102D7000F0000020B4170020280A000040130020B3
:102D8000E02E00008813000000120020F0B52A4C4D
:102D90008BB020700E462A4828490160294981607D
:102DA000294941602949C1602949016129492A4DC0
:102DB000816129688847F0B22849607048432849F2
:102DC0004018E968884700242648089001200490AC
:102DD000042608200594069407940196029603940D
:102DE00000900123EF69224610211846B8470120C0
:102DF000069407940894099400940294039404940C
:102E0000019605900423AE6908220146B0472021AF
:102E10006A6D01209047402002F0D0FD0120002380
:102E2000024600901946022002F01AFC04481C30A9
:102E3000846000200BB0F0BDF00000204540000889
:102E400098170020713E0008CD4000088D3F000813
:102E5000F53E0008613E00082C7800085016080076
:102E600060BDAA19B80B000010B50B480078002807
:102E700003D00120FFF7D6FD0CE00848416BFA2093
:102E80008847074C0220A060FDF7E2FF6062FDF773
:102E9000DFFFE061002010BDF00000202C7800086A
:102EA000B417002030B583680122134002D00022FD
:102EB000104630BD8C684B68C9682343C468034D15
:102EC0002C4021430B43C360F2E70000C73FFFFFE4
:102ED00030B583680122134002D00022104630BD75
:102EE00018C94D6823430C6889682C4323430B435E
:102EF000C168024C21400B43C360EFE73CC2FEFFB8
:102F000008B504494A6902434A6149690140009190
:102F100008BD00000010024008B50449CA69024318
:102F2000CA61C9690140009108BD0000001002405B
:102F300008B504498A6902438A61896901400091A0
:102F400008BD00000010024070B5094E044671181B
:102F50002039049D0C34CE7F0830102D03D0325020
:102F6000C87F035170BD3251C97F0B5070BD000046
:102F700050730008044A51182039C97F425852083A
:102F8000520042507047000050730008044A511824
:102F90002039C97F425801231A434250704700002C
:102FA00050730008044A51182039C97F425802233F
:102FB0001A4342507047000050730008054B10B58B
:102FC00059182039C97F435803242403A3431343CA
:102FD000435010BD20780008054B59182039C97F8F
:102FE000001D0B581B0C1B0413430B5070470000B3
:102FF00050730008054B10B559182039C97F435844
:10300000034C23401343435010BD000020780008B8
:10301000EFBFFFFF054B10B559182039C97F435842
:103020008024A3431343435010BD000020780008C0
:10303000054B10B559182039C97F43580324A40201
:10304000A3431343435010BD20780008054B10B52F
:1030500059182039C97F43582024A34313434350B0
:1030600010BD000020780008054B10B55918203914
:10307000C97F43584024A3431343435010BD00006D
:1030800020780008054B10B559182039C97F4358DE
:1030900003242402A3431343435010BD20780008A7
:1030A000F0B500243EE001232A46A3401A4038D060
:1030B0004F680668134653435D005D19AE435F4396
:1030C0003E4306604E68012E01D0022E05D18F6866
:1030D00086685F43AE433E4386600F69C668AE4371
:1030E0001D467D432E43C6604D68022D19D1FF2A2F
:1030F0000AD84E69056A534353431A01D21A9543BD
:1031000073431D4305620CE0130A1A465A435A439F
:103110005A4313019E1A4D69436A6A43B3431343EA
:103120004362641C0A681546E240BCD14A68012A21
:1031300001D0022A06D1CB6841682A4691435A43FE
:10314000114341600120F0BD10B5044601F012FCAE
:10315000206001F0F5FB606001F000FCA06010BD94
:10316000014610B5002000290FD110490A6B9207C3
:10317000920F012A0AD0022A11D0032A09D001F0A5
:10318000F9FB01F0DDFB01F0E9FB10BD01F0F2FB02
:1031900010BD09688907C90FFAD0054810BD096A32
:1031A0008907C90FFAD00120C00310BD00100240EA
:1031B00000127A0010B5036800225B06DB0F25D1F0
:1031C0000CC98C681A434B6823431A43CB681A43D3
:1031D0000B691A434B691A438B691A4303680C4CF9
:1031E00023401A43026042680A4B1A40CB681B0C0A
:1031F0001A430B681A43426001238A695B0308394A
:103200009A4202D1898C89B201610122104610BD17
:103210004000FFFFFBF0FFFFF0B50268194B1A4CAE
:10322000984201D0A04203D17025AA434D682A4399
:10323000164D174E174F98420AD0A04208D0164C90
:10324000A04205D0A84203D0B04201D0B84204D178
:1032500003242402A243CC68224302608A68C2622B
:103260000A888262984205D0A84203D0B04201D0B9
:10327000B84201D1097C01634169012211434161D6
:103280001046F0BD002C0140000400400040014009
:1032900000440140004801400020004041680122F4
:1032A000D202914341608168082291438160704756
:1032B000FEB5044600680D460026C007C00F43D186
:1032C000E9686868AA6908432969114308432168C5
:1032D0001E4A114008432060A96860680322120357
:1032E0009043084360606969A068121190430843E5
:1032F000A0601748844203D10020FFF731FF06E0A9
:103300001448844220D16846FFF71EFF0298002827
:103310001AD02968002917D00126AA69F3039A4216
:103320000CD140004A088018FCF7DEFE81B20A4842
:1033300008400907490F0143E16005E04A081018F9
:10334000FCF7D2FE80B2E0603046FEBDF369FFFFBD
:103350000038014000440040F0FF00000348012213
:103360004169520351404161704700000008004824
:1033700010B580220249FCF718FF002010BD0000A4
:1033800090770008F0B584461948184D836812C834
:103390000022184F0AE0A85BB84206D17019408895
:1033A000A04202D904461146531C521C012056016A
:1033B00080028642EFD30E4E01207460B36031600C
:1033C000002906DB480141192022604601F01CFF5C
:1033D00001E061468880B068012140018902203007
:1033E000884201D90020B0600020F0BD00C800086C
:1033F00098000020AA5500001FB50B46024604A104
:10340000684603F01DF90146684601F077FA1FBDD2
:10341000201B5B25643B25644800000070B501203B
:103420008AB04002FFF784FD224CA06A0326304395
:10343000A0622149B0050A68824302430A60A26A79
:1034400083111A43A2620A68824302430A6000257C
:1034500005950695079505A920460895FFF722FDD5
:103460000120039000950195029569460495204638
:10347000FFF72EFDE06804218843E0606069C00822
:10348000C000304360616068084360606068082184
:1034900088436060A06817218843C9070843A0607B
:1034A000A068C00FFCD1A06804490840401CA0607F
:1034B0000AB070BD0024014008270140E8FFFF7FEB
:1034C00010B50120FFF71CFD00210A2000F084FC4C
:1034D0000A2000F077FC00210B2000F07DFC0B207F
:1034E00000F070FC10BD0000F0B5012087B0400472
:1034F000FFF706FD01208004FFF702FD0120C00454
:10350000FFF7FEFC01208005FFF7FAFC0126C02032
:10351000002403256A46049631C20927FF0669463E
:103520003846FFF7BDFD8020694631C169463846FF
:103530000494FFF7B5FD93200001009003946946C1
:103540000196029504943846FFF7AAFD3002B8614F
:1035500068026A46049631C269463846FFF7A0FD04
:1035600021486A46049631C269462048FFF798FD13
:103570001F480090039469460196029504941B48E5
:10358000FFF78EFD072040030090029403946946E4
:10359000019604941748FFF783FD80206A4604963D
:1035A00031C269461148FFF77BFD30036A46049635
:1035B00031C269463846FFF773FDF003009003946B
:1035C00069460196029504943846FFF769FD40204C
:1035D0000090039469460196029504940348FFF70E
:1035E0005FFD07B0F0BD00000704000000040048C4
:1035F000EEBC000000080048084907480860084879
:1036000008600420486007488860CA685207FCD1F7
:103610000861054808607047CCCC000000300040CD
:1036200055550000FF0F0000AAAA0000F0B591B0A8
:10363000282106A8FCF7D2FD18216846FCF7CEFD2C
:1036400001252D032846FFF773FCA801FFF758FC5E
:103650000024082002260327039404946A46059454
:10366000C1C269461F48FFF71BFD1020694603943D
:10367000C1C101200490694605941A48FFF710FD66
:103680002020039404946A460594C1C269461548F3
:10369000FFF706FD0021192000F09EFBFF200530FA
:1036A00007900720000208900694E8100B900994F8
:1036B00008200A940D940E940C9007200A4C0F9049
:1036C00006A92046FFF776FD6068102188436060F8
:1036D0006068A84328436060206840210843206058
:1036E00011B0F0BD0004004800300140F0B591B0C9
:1036F000282106A8FCF772FD18216846FCF76EFD2C
:103700000127BF033846FFF707FC3801FFF7F8FB36
:103710000024781002250326039404946A46059435
:1037200061C269461C48FFF7BBFC009703940494F0
:1037300069461948029601950594FFF7B1FCA80364
:10374000039404946A46059461C269461248FFF7DF
:10375000A7FCFF2005300790072000020890069480
:10376000099428020A940C940D940E940B9007204F
:103770000A4C0F9006A92046FFF71CFD6068102137
:1037800088436060606808210843606020684021C9
:103790000843206011B0F0BD00040048003800402C
:1037A00010B586B014216846FCF718FD1020FFF70D
:1037B000B3FB0021112000F00FFB112000F002FBF1
:1037C0002F2069460880002001900848084C02908C
:1037D0002046FFF721FD2068802188432060E068B3
:1037E00001210843E06006B010BD0000E7030000BF
:1037F0000010004070B501208EB08003FFF798FBE9
:103800000320400207900220089003200024099022
:10381000012509200A9407A90C950B94C006FFF70F
:103820003FFC3A4E102202213046FFF7E3FB002214
:1038300002213046FFF7C2FB002202213046FFF78B
:1038400005FC002202213046FFF70EFC80220221F7
:103850003046FFF7DFFB002202213046FFF712FC63
:10386000002202213046FFF7E3FB0022032130460D
:10387000FFF7C0FB002203213046FFF79FFB002229
:1038800003213046FFF7E2FB002203213046FFF719
:10389000EBFB802203213046FFF7BCFB0022032113
:1038A0003046FFF7EFFB002203213046FFF7C0FB55
:1038B00000211B2000F090FA1B2000F083FA14482E
:1038C000694600680090019402940394059406945C
:1038D0000C20104C04902046FFF7EAFC6068290594
:1038E0000843606060684900032252059043084322
:1038F0006060A06849120843A0602046FFF7CEFC34
:103900002068284320600EB070BD00000000024017
:10391000340000200038014070B58EB01C2168468C
:10392000FCF75CFC182107A8FCF758FC0124640490
:103930002046FFF7F1FA2046FFF7E2FA0E20079043
:1039400002200890032001250990002409200A95EF
:1039500007A90C950B94C006FFF7A2FB414E10225D
:1039600004213046FFF746FB002204213046FFF7D2
:1039700025FB002204213046FFF768FB00220421CA
:103980003046FFF771FB802204213046FFF742FBEF
:10399000002204213046FFF775FB00220421304647
:1039A000FFF746FB002205213046FFF723FB0022EC
:1039B00005213046FFF702FB002205213046FFF7C4
:1039C00045FB002205213046FFF74EFB80220521F2
:1039D0003046FFF71FFB002205213046FFF752FB60
:1039E000002205213046FFF723FB00211C2000F0B8
:1039F000F3F91C2000F0E6F9A61EFF21304600F086
:103A0000EBF9304600F0DEF91748EE03006800904D
:103A10000194029403940C2004AA51C2134C6946E9
:103A20002046FFF745FCA06821140843A060A06869
:103A3000B0433043A06020681F21490588430843F4
:103A4000206020684911884308432060A068A114C1
:103A50000843A0602046FFF721FC2068284320602F
:103A60000EB070BD0000024038000020004400404D
:103A700000B50846042A02D80020C04300BD0178E2
:103A80007F2902D90120C04300BD41784906490E73
:103A90001F2902D90220C04300BD114603F0FCF8E3
:103AA0000028F9D0042000BDF7B58EB00F46109A5B
:103AB0000E98FFF7DDFF002803D00020C04311B0AF
:103AC000F0BDBC49387809783A46884201D00020D8
:103AD000F5E750785388BA885DBA56BAB64A0224D8
:103AE0001170507029050A0E2907090F030002F012
:103AF000D2FD11C60A5995ADC7E5C6C6C6C6C6C62B
:103B0000C6C6F3F1C600F01DC008AB49019088702D
:103B1000002041E000200590012004900798002734
:103B2000C0000A902EE0290701222809090FD202BD
:103B300095420FD24200A1481218092080011018A6
:103B4000808EFDF7E3F8002812D005990498014310
:103B500005910DE0420099481018FF308130808AAD
:103B6000FDF7D4F8002803D0049905980843059080
:103B700004986D1C4006000E7F1CADB20490082F07
:103B800003DA0A98C019B042CDDB8B4A0799059831
:103B90005118C8700798401C019907908842B9DBFA
:103BA00064186BE0F01DC008834901908870002004
:103BB0002FE0002005900120049008980027C00005
:103BC0000A901CE02805000E42007C4829071218C4
:103BD000092080011018090F808AFDF797F8002846
:103BE00003D0049905980843059004986D1C40067D
:103BF000000E7F1CADB20490082F03DA0A98C0199A
:103C0000B042DFDB6C48089A05998018C1700898AB
:103C1000401C019908908842CBDBC1E772006649DD
:103C200000208A700FE02B185F00644BFF180923F7
:103C3000DB01FB189B8E47009C461B0A7F18FB701C
:103C400063463B71401CB042EDDB16E072005A49FE
:103C500000208A700FE02B185F00584BFF180923D3
:103C60009B01FB189B8A47009C461B0A7F18FB7030
:103C700063463B71401CB042EDDBA418641C8AE033
:103C8000002E12D0FF200002864207D14B4852007E
:103C900012189D208000101802F00EF83946464890
:103CA000109AFCF782FA109A7FE0444852001218EA
:103CB0009D208000101801F0F5FAEFE73979787946
:103CC000090201433D486A0012180920C00110187A
:103CD0008186E3E742E0FFE7F01DC0083649019026
:103CE0008870002035E03818C079059001200490D4
:103CF00000200A900B98C0000D9024E029070122B3
:103D00002809090FD2029542059B049A07D21A404E
:103D100043002A481B189D208000181805E01A400F
:103D2000430026481818FF30953001F0D9FF049859
:103D30006D1C4006000E04900A98ADB2401C0A901B
:103D4000082804DA0D980A994018B042D6DB0B987F
:103D5000401C0B9001998842C5DB12E000200EE068
:103D60004100CA19D179127A090211432A18530065
:103D7000124A9B180922D2019A189186401CB0421F
:103D8000EEDB0D48B9788170F978C170397901712D
:103D900079794171241DA1B2074802F07DFF0649DF
:103DA0000855000A09194870A21C03490E9801F031
:103DB00067FF8CE690000020B80A0020C00D0020AC
:103DC00070470000C106C90E012088400149086003
:103DD0007047000000E100E08307FF22DB0E9A40FD
:103DE0008907090E994000280BDA0007000F0838F0
:103DF000830808489B001818C36993430B43C361A9
:103E00007047830804489B001B18186890430843B8
:103E10001860704700ED00E000E400E08307FF2237
:103E2000DB0E9A408907090E994000280BDA00073B
:103E3000000F0838830808489B001818C36993438B
:103E40000B43C3617047830804489B001B18186824
:103E5000904308431860704700ED00E000E400E084
:103E60000248016D491C016570470000B41700202D
:103E7000FFB581B004461B490298888116461F464B
:103E800021461948029AFCF790F916482146343029
:103E9000029AFCF78AF91548006B8047144C002001
:103EA0006179002900D060710F4D943D6860FCF786
:103EB000CFFF6969401A2863E67028462771603091
:103EC000067247722869401C2861207802990028F0
:103ED000607803D0FEF72CFD05B0F0BDFEF706FEBE
:103EE000FAE70000C0140020481800202C780008D1
:103EF000F000002070B51F4C1F49A06C1F4D401CE6
:103F0000A064088A401C088201206871FCF7A0FFA9
:103F1000A16A401AE0622878002822D1A06B401CD8
:103F2000A063E06B401CE063216C884200D92064F0
:103F30001349012802D9FF22F5328A64022811D0E0
:103F4000104A032800D98A6404280FD0062803D910
:103F50008A640D4A0021D182072802D1606E401C7C
:103F6000606670BDE06D401CE06570BD206E401C59
:103F7000206670BDB4170020C0140020F00000209F
:103F800040130020881300000012002070B5264C5A
:103F90000025264EA560306B8047FCF759FFA16ACB
:103FA000401AE062FCF754FF2149A062C889401C16
:103FB000C881A06B401CA063E06B401CE063216CD7
:103FC000884200D920641B49012802D9FF22F5321A
:103FD0008A6402280DD0184A032800D98A6404286C
:103FE0000BD0062802D98A641449CD82072808D04C
:103FF0000AE0E06D401CE06506E0206E401C206693
:1040000002E0606E401C60660D48007800280AD10E
:10401000716BFA2088470220A060FCF719FF6062EC
:10402000FCF716FFE06170BDB41700202C78000883
:10403000C01400204013002088130000001200204C
:10404000F000002070B51B4C00201B49A0600889BF
:10405000401C0881FCF7FCFEA061FCF7F9FE174D3F
:10406000A062286B80471648696B0078002801D051
:10407000502000E0FA2088470220A060FCF7E8FE0C
:104080006062FCF7E5FEE0610E480122416992039F
:1040900051404161FCF7DCFE0B494A6E821A8A6688
:1040A0004866C86E824200D2CA66086F824200D952
:1040B0000A6770BDB4170020C01400202C780008D7
:1040C000F0000020000800484013002010B5064C06
:1040D0000020A060FCF7BCFEA062606C401C606425
:1040E0000248006B804710BDB41700202C780008F0
:1040F00010B501200449C006486004480168491C05
:10410000016000F005F810BD00ED00E03000002077
:1041100070B5094CE06F00280CD0084D084902200A
:104120002A68FDF7A9FE00202860E0678021044886
:1041300002F07EF970BD00007403002040000020F2
:104140008804002010B50648054B00780021403B4C
:104150005A1840325478491C14700F29F8DB10BDEE
:10416000000E002010B5084C084B01220221A06D62
:10417000FCF7C6FB064801F047FDE06D401CE0651A
:10418000A06D2066002010BD4013002039300000D3
:10419000741500200248C16D491CC165002070479C
:1041A00040130020F3B5FE4E89B03068002870D06F
:1041B000706800281CD000220D21082001F0A6FD07
:1041C00000221146082001F0A1FD0122114608201D
:1041D00001F09CFD0020F34F01463A184032401C8C
:1041E00011701028F9DBEF4D0024012140358AE2DF
:1041F0000122E1E7A2000998099B805CD31805938E
:104200005A78009201265B8801931B2873D012DC38
:104210000246030002F03FFA1B5C72727272727205
:104220003E3E3E3E3E3E5C5C5CA7A7A73E3EBEBE19
:10423000BEBEBEBE5C00342870D011DC01461C3905
:104240000B0002F028FA18A7A7A7A7A7A7A7A7A758
:10425000A7A7454545454545454545454545FC4593
:104260003A2873D008DC014635390B0002F013FA06
:1042700005E76E56E76E3000DC2804D004DC3B28EE
:10428000EFD0C82824D128E1DD28FCD0FA28F9D1C4
:1042900023E141E2D01F030002F0FDF90E080A10ED
:1042A000181B1D1A1A1A1A1A1A20261A287C4AE0F4
:1042B000FFF748FF00281FD0287C3AE0FFF742FFB5
:1042C000002816D1287C002813D125E000F0D0FA70
:1042D00002E22878F7E7FFF735FF1DE0287C002889
:1042E0000AD0002905D007E0287C002804D1002945
:1042F00002D0012010E04DE000200DE0130002F09C
:10430000CAF9070C050E111B262E0C0000F0B0FA9E
:1043100001990098FCF70EFD2874DDE120E100F022
:10432000A7FA0CE0287C0028E6D001990098FCF759
:1043300001FD0028E0D0DCE7287C0028DCD00199D2
:104340000098FCF7F7FC0028D6D1D2E761E1287C81
:104350000028CED101990098FCF7ECFCB3E7287C4B
:104360000028ECD0C5E7102804D0112804D0122A68
:10437000AED10AE02A7C03E0287C0028A8D00122E4
:104380000199009801F0C2FCA6E1287C00289FD08A
:104390000022F5E70599029115380E79030002F025
:1043A0007AF9120A1215181B0F1E3E4F5F6F2E7FEF
:1043B000878B8F93839A00F05BFA13E028748AE06E
:1043C00000F056FA1EE000F053FA2BE000F050FA2D
:1043D00039E000F04DFA46E000F04AFA53E0287C5C
:1043E000002876D030460199FCF738FD0646029841
:1043F000C1884079FCF732FD864268D069E0287CAC
:10440000002866D030460199FCF728FD0646029840
:10441000C1884079FCF722FD864258D159E0287CBA
:10442000002856D030460199FCF718FD0646029840
:10443000C1884079FCF712FD864248DB49E0B3E0D1
:10444000287C002845D030460199FCF707FD064638
:104450000298C1884079FCF701FD864237DC38E0DC
:10446000287C002835D030460199FCF7F7FC064639
:104470000298C1884079FCF7F1FC864227DD28E0EC
:10448000287C002825D030460199FCF7E7FC064639
:104490000298C1884079FCF7E1FC864217DA18E0FF
:1044A000287C002813D19DE7287C00280FD1A9E79C
:1044B000287C00280BD1B5E7287C002807D1C2E76B
:1044C000287C002803D1CEE7287C0028DBD00120FF
:1044D00074E7002072E70226FEE005991646097986
:1044E0000091C8280CD0DC2821D0DD2827D0FA285C
:1044F000F1D1F000C0194030007EC00627D507E09A
:10450000F000C0194030007EC00601D400211FE039
:10451000287C002820D001990098FCF79FFC0146D8
:10452000304600F0C7FE304600F0FAF846E7F000EB
:10453000C0194030007EC006EAD4012108E0F00036
:10454000C0194030007EC006E2D4022100E0032101
:104550003046FDF797F9DBE7304601F0EBFDE2E787
:104560000599022609790091342802D0372816D1FE
:1045700008E0287C002812D001990098FCF76EFC16
:10458000401C07E0287C002809D001990098FCF71E
:1045900065FC401E02460199009801F02DFC9BE04D
:1045A000380B0020C00D0020059933280A790092AD
:1045B0004A790392C988029114D035281BD0382833
:1045C00089D1287C002886D01046FCF747FC064697
:1045D00001990098FCF742FC321A0299039801F005
:1045E0000BFC78E7287C0028FBD001990098FCF7A9
:1045F00035FC0246F1E7287C0028F2D001990098AA
:10460000FCF72CFC064602990398FCF727FC3218AD
:10461000E3E7059936280A794B790593CB88079308
:104620004B7A03934989029106D0392812D03A284F
:1046300020D03B284FD132E0287C00284BD01046B8
:104640000199FCF70BFC064607990598FCF706FC58
:1046500032180CE0287C00283DD010460199FCF768
:10466000FDFB064607990598FCF7F8FB321A0299FC
:1046700003982EE0287C00282DD010460199FCF7E5
:10468000EDFB06B207990598FCF7E8FB00B246433C
:1046900032460299039801F0AFFB321416E0287CF1
:1046A000002818D010460199FCF7D8FB06B20799EC
:1046B0000598FCF7D3FB01B23046FBF72BFD02B2A5
:1046C0000E460299039801F097FB3246029903982F
:1046D000491C01F091FB0326201141000F482307DC
:1046E00008181B0F0121028999408C46114000D007
:1046F00001212B7C0830002B634601D01A4300E0D7
:104700009A430280A4190A98844200DA72E50348A9
:104710004168491C416000200BB0F0BD380B0020FF
:10472000FEB50746402802DB0020C043FEBD2C48F2
:10473000F9000E1800964036348BE10601D40020B3
:10474000FEBDA1063CD561063FD426490968009804
:104750000A25406D0190081AA1070FD0A107890F03
:10476000012905D0022905D0E143890705D005E0DC
:10477000642503E07D25ED0000E01B4DA84224DB0D
:104780002946FBF7C7FC014615487A0012180B2092
:10479000800110188446808E019B401869435B1885
:1047A000009980B24B650D2189015118898E814293
:1047B00003D8084640210C4334836146888604E0D0
:1047C000600602D5402084433483307EB9B240066F
:1047D000C20F052001F09AFA307E4006C00FFEBDE0
:1047E000C00D0020DC01002010270000F7B50546B1
:1047F000FCF703FB044602992868A142A96806DC7D
:104800004018029A0199FBF7D0FC029919E0401870
:1048100022460199FBF7C9FC21462846FCF7B2F86D
:104820002846FCF7EAFA06460298071BB7420DDC59
:10483000A96828683A46401801990919FBF7B5FCA0
:1048400039462846FCF79EF80298FEBD002E0CDD86
:10485000A96828683246401801990919FBF7A5FC98
:1048600031462846FCF78EF8A4192046FEBD00000C
:10487000074A0F2011183F235B5C4031401E0B702C
:104880000028F7DC02494031087C087070470000BE
:10489000C00D002000B500F001F800BD70B572B683
:1048A0000122134B12039A611249040A0C7300246B
:1048B0008D68AD07ED0FFBD00F4D6C62002400E05A
:1048C000641C8E683606F60FFAD108738868800774
:1048D000C00FFBD000206C6200E0401C8C682406F6
:1048E000E40FFAD1E8629A629A6162B670BD000084
:1048F0000004004800380040C013002010B50C46EA
:104900000A4601460348FFF771FF01F079FD204692
:1049100010BD00003803002010B50C460A460146C1
:104920000348FFF763FF01F06BFD204610BD000058
:104930003803002010B50C4601F0CAFD204610BD1A
:1049400004494968F0221140034A0909515CC840F2
:1049500070470000001002404C7900080349496884
:10496000034A4905490F515CC84070470010024096
:104970005C79000810B5064841680C2001400548E4
:1049800005D0042903D0082901D100F005F810BD95
:104990000010024000127A0010B50C4C6168012230
:1049A00012040B48114002D0914200D14000E16A4C
:1049B0000907090F491CFBF797FB61680F22920456
:1049C0001140890C891C484310BD000000100240B2
:1049D00000093D0001207047F7B5002415460F4639
:1049E000012A02D0094E0A4809E00A4E0A4806E0A8
:1049F00000993246095DFCF731F8641CE4B2BC4210
:104A0000F6D3012D01D0C04380B2FEBD21100000BD
:104A10000F1D000005800000FFFF000010B500F032
:104A2000DFFC032804D0042803D0052803D000208D
:104A300010BD022010BD012010BD032070470000F2
:104A400010B50E4C20610E4800F05AFD002000F019
:104A5000CBFF012000F03BFF0021084600F0EAFDFB
:104A60000421002000F0FCFF064800231A460146FE
:104A700000F039FE0020A07010BD0000F8000020FA
:104A8000A94B0008FFFF0000F8B501200003092131
:104A9000C90609698843002100286CD1364CA170F1
:104AA00000F094FC0546354800F086FCE80706D087
:104AB0002069002803D00068002800D080476806DD
:104AC00006D52069002803D00069002800D080475F
:104AD000A80723D5FF226946294800F0CDFC2848C5
:104AE000143800F085FC2069002817D08668002E55
:104AF00014D0234814380178012902D0002905D0A8
:104B00000CE00D230C22C356825603E00623052237
:104B1000C3568256684601781948B04728060AD518
:104B20002069002807D08169002904D0E843C00526
:104B3000C017401C8847A80514D500F051FC042874
:104B400004D000F04DFC052805D00BE020690028BA
:104B500008D0406803E02069002803D0C06800281E
:104B600000D08047A80606D52069002803D0006938
:104B7000002800D08047F8BDF8000020FFFF0000AB
:104B80007C18002070B50C46012500F0A3F82046E3
:104B900000F0A4FE002000F033F80120FCF7EEF94D
:104BA00000F04AFA284670BD01490120887070471C
:104BB000F800002070B50025012000F08BF80020DF
:104BC00000F0B8FE00240120FCF7D8F900F06AFCE0
:104BD000C007C00FA040641C0543E4B2202CF2D3F0
:104BE00000F02AFA284670BD10B500F0DCFC10BDBC
:104BF00010B500F0E0FC10BD10B500F053FC10BD86
:104C000010B50446074800231A46014600F06BFD24
:104C100005484078002801D0044800E0A00100F0D9
:104C200089FE10BDFFFF0000F8000020FFFFFF001D
:104C300010B50446074800231A46014600F053FD0C
:104C400005484078002801D0044800E0A00100F0A9
:104C500083FE10BDFFFF0000F8000020FFFFFF00F3
:104C600070B505460C480C4600231A46014600F074
:104C70003AFD00F0FBFB01460848012909D0047207
:104C8000064800F0B5FD00222146284600F0CAFC87
:104C900070BDC473F4E70000010200007C1900201D
:104CA00010B500F01BFE10BD10B5084B084A0128D6
:104CB00008D0D079012804D119701172044800F08D
:104CC00097FD10BD1970D173F8E70000F8000020BF
:104CD0007C19002010B50A4C012805D0002000F0F6
:104CE000E1FD0020607010BD012000F0DBFD617867
:104CF00020788142F7D0607000F004F810BD000009
:104D0000FB00002070B504460B480470447001207D
:104D1000FFF7E0FF1D208001451C002C04D034214A
:104D200000F04BFF442103E0142100F046FF242152
:104D3000284600F042FF70BDFB000020FFB583B0A5
:104D400016460D46654A15990D9F109B51700F9997
:104D5000002902D011460B7002E06049FF220A7060
:104D60005F4902910C46083C002816D001287CD1EE
:104D7000002000F04BFE0E98C0B200F0D5FC0121DF
:104D80002172F2B257482276405D60760698A0768E
:104D9000002D77D0012D77D078E0002000F036FE8E
:104DA000002020724E482838C6620B202075002D46
:104DB0000ED04C490020091DC2008B58AB425CD874
:104DC00052189268AA4258D9C0004018007B00E0EF
:104DD0001F2060754248002128380170FA00428087
:104DE000042202711822427181710F9B01225340EB
:104DF0003A4DC3712B780372119B002B00D0F22225
:104E00004272817200F084FC207A002800D00120D8
:104E1000FFF760FF029800F08FFC3148283800F05F
:104E2000E7FC31A003C800900191684600F0F5FD51
:104E30002F4800F055FE3046FBF7A2FB02460B461A
:104E400000202C49FBF7FAFA0322FBF76FFB04461C
:104E50000E460E98FBF794FB22463346FBF786FA84
:104E60000022254BFBF782FA02E004E00AE00BE0A7
:104E7000FBF794FBE86007B0F0BD401CC0B21528FA
:104E80009AD3FEE70B2E0BD00C2E09D00020E07633
:104E9000134828380170052A04D0062A02D006E0FB
:104EA000E176F5E70C2F02D20C21818100E08781A9
:104EB0000F990A4C81732178C17311990174149967
:104EC00041740120FFF706FF029800F035FC04480A
:104ED000283800F08DFC0948E060CCE7F80000209D
:104EE000A419002098780008C194C10000000000B7
:104EF000FF0100000000F03F00408F40FFFF000076
:104F000010B500F043FD10BDFFB5404983B00C461D
:104F100028340C9E02940E9F0125083C002802D0E4
:104F200001286BD132E000202072CE620B2626755C
:104F300063750A630870FA004A8004220A71182215
:104F40004A7188710F986840C8711098002802D083
:104F5000F220487200E04D728D7200F0D9FB207A89
:104F6000002800D00120FFF7B5FE029800F0E4FB16
:104F7000264800F03DFC26A103C900900191684637
:104F800000F04BFD244800F0ABFD37E02572F0B295
:104F9000224A2076D25C62760D9AA276002B02D04D
:104FA000012B02D003E00B2E09D00C2E07D00022DB
:104FB000E2760D70052804D0062802D006E0E576DA
:104FC000F7E70C2F02D20C20888100E08F810F9828
:104FD000887313480078C87310980874139848743D
:104FE00000F096FB207A002800D00120FFF772FE27
:104FF000029800F0A1FB054800F0FAFB049800F0CD
:1050000093FC07491498886007B0F0BD7C19002014
:10501000C194C10000000000FF0100009878000862
:10502000F800002010B50C4600F058FC204600F0B7
:105030007BFC00F00DFD10BD08B500206946009016
:1050400008780421084369460870009800F0BEFC07
:105050000220FBF793FF08BD10B500F059FB10BD0F
:1050600010B500F0F1FA10BDF3B502460020574923
:105070008BB0002A55D0012A7ED10F462037787E8A
:10508000534A800180183C7E0C22121BD2008018EB
:10509000C21FF93A10464668084615688089FBF732
:1050A0006FFA00224B4BFBF7AFF82A463346FBF76B
:1050B0005DF907910690B87E8007800F001DFBF711
:1050C0005FFA05910490F87E002800D00220201A93
:1050D0008000FBF741FA07460C980391C000A1003D
:1050E000411A3A48027C807B12018918012852D06B
:1050F0000020081A1C30FBF72FFA3A46039BFBF7F7
:105100009DF901F025FD059B049AFBF72FF900227C
:1051100007460C461346FBF75FFA3ED23846214657
:105120003DE00C46C86AFBF72BFA06460F460C9882
:10513000FBF726FA0D46069061796088C908401889
:10514000FBF71EFAE279002A1ED00022224BFBF761
:105150005BF82B46069AFBF757F8627A022A16D0BC
:1051600000221346FBF750F80322FBF7DFF9324623
:105170003B46FBF763F900E025E00022174BFBF705
:10518000F5F802F0D9F81CE000221346DFE7002210
:1051900001239B07E6E71420ABE70020014600222D
:1051A0000F4BFBF731F82A463346FBF7DFF8079B36
:1051B000069AFBF729F80B4A0B4BFBF725F801F091
:1051C000BBFDFBF7EBF90DB0F0BD00007C19002032
:1051D00010010020000011400000F03F00408F400F
:1051E000000020402B8716D9CEF7EF3F10B500F016
:1051F000E4FC10BD10B500F0E6FC10BD00B50820C1
:10520000FCF79AFBC0B200BD70B5D4170346A40FDB
:105210000020A418A41003E085004E595E51401CE4
:105220008442F9DC6000D40FA418641003E0450048
:105230004E5B5E53401C8442F9DC104670BD00B5E5
:10524000FFF7DCFF00BD0000F8B500228024D24348
:10525000114D00218C4623464B435B191F880F4E8E
:10526000B74209D17E26F75A0D4EB74204D15B886A
:10527000634501DD0A469C46491C0829EBDB082AE8
:1052800005D2624351198022FFF7BEFF01E0FEF70D
:105290006FF80020F8BD000000C00008AA5500000B
:1052A000A55A00000B0702881B0F012199408A4371
:1052B0000280704730B5402802DB0020C04330BD7B
:1052C0000D4BC200D21814464034257EAD0611D4D1
:1052D0004000C0180D239B01C31899860B230021A1
:1052E0009B01C0188186054800685065208B2021ED
:1052F00008432083002030BDC00D0020DC010020C9
:1053000010B500F001F810BD03488168C907C90F46
:1053100000D0C068704700000030014070477047FF
:1053200070470000174908B5884204D9E121684652
:105330000170E9211EE01449884204D9D72168464A
:105340000170D82116E01149884204D9C12168466C
:105350000170C5210EE00E49884204D975216846C6
:105360000170812106E00B49884204D96B2168460F
:1053700001706F21417002226946982000F000FC04
:1053800008BD000000E9A43580F8A9328044E52D6D
:10539000000B6B1B40FC541910B5064840780028E0
:1053A00001D0062803D100F0BDFBFFF7B9FF00F0E4
:1053B000B1FB10BDD001002008B5020A69460A7091
:1053C00048700222104600F0DBFB08BD08B502223F
:1053D0006946122000F0C8F86846008840BA08BD47
:1053E0000148407870470000D0010020022070473B
:1053F00038B5044603226946142000F0B5F81A496E
:1054000088782070002808D0012816D01421204662
:10541000FAF7E4FE0F20207038BD6846007820714E
:105420006846407840424010A0716846807840420B
:10543000401060710020A06038BD6846007840428E
:105440004010207368464078802801D2800802E02E
:10545000FF38013880106073684680784042401001
:10546000A0734868206138BDD001002001488078D1
:1054700070470000D0010020F8B50C460646002019
:10548000694608701546204600F018F82278AA42AE
:1054900001D90120F8BD68463146007800F042F895
:1054A0000020F8BD08B501226946152000F05CF81F
:1054B000684600784042401040B208BD38B50D46FD
:1054C000044602226946132000F04EF80A4880780C
:1054D000012809D1094800F066F8C00904D007483E
:1054E000801E00F060F801E0684600782070684691
:1054F0004078287038BD0000D0010020040700006B
:1055000010B500F07DF800F00DFB002000F06CFA03
:10551000012000F0E1F802490120487010BD0000B0
:10552000D0010020F7B516460446FFF735FF0125E8
:10553000ED030927FF06BD621E2000F081FD204615
:1055400000F07EFD002000F07BFD002406E000203E
:1055500000F076FD01990855641CA4B2B442F6D35C
:10556000BD6100F0D7FAFEBDF7B516460446FFF759
:1055700013FF0125ED030927FF06BD62204600F059
:105580005FFD002000F05CFD002406E0002000F03C
:1055900057FD01990855641CA4B2B442F6D3BD610D
:1055A00000F0B8FAFEBD08B50122694600F003F824
:1055B0006846007808BDF7B516460446FFF7ECFECE
:1055C0000125ED030927FF06BD621D2000F038FD0F
:1055D000200A00F035FDE0B200F032FD002000F0BE
:1055E0002FFD002406E0002000F02AFD0199085557
:1055F000641CA4B2B442F6D3BD6100F08BFAFEBDC8
:1056000010B50A20FBF7BAFC054C4020A06214201C
:10561000FBF7B4FC4020A0610A20FBF7AFFC10BDF3
:105620000004004810B5144600F04AF9204600F086
:10563000FDF910BD08B56A46107051700222694626
:105640008F2000F09DFA08BD10B500221146C5203C
:1056500000F096FA01490720487010BDD0010020E3
:105660007CB56C46069D20706170A270E370280CBA
:105670002071280A6071A57105226946882000F012
:105680007FFA0249072048707CBD0000D00100204D
:1056900008B5020A69460A704870044880780028F4
:1056A00003D10222024800F08EFA08BDD00100208A
:1056B000BE06000008B5020A69460A704870044830
:1056C0008078002803D10222024800F07CFA08BD4D
:1056D000D0010020BC06000001B5012269469D20D2
:1056E00000F04EFA08BD7CB5050A6C462570607066
:1056F000080AA070E170100A20716271180AA07186
:105700000822E3716946104600F03AFA7CBD0000B9
:1057100010B500221146C12000F032FA01490320E1
:10572000487010BDD001002001B501226946A020BB
:1057300000F026FA08BD00007CB504460020009069
:105740000190224920788978884201D000F0AAF897
:105750002078002810D001280DD1217C68460170E6
:10576000617C4170A17C8170E17CC170042269463A
:105770008B2000F005FA7CBD08256068FAF700FF71
:1057800002460B4600201249FAF758FE0522FAF7A6
:10579000CDFEFAF703FF020C69460A70020A4A704E
:1057A0008870207BC870607B0871A068FAF7E8FEFB
:1057B0000022084BFAF742FEFAF7F0FE020C6946A7
:1057C0004A71020A8A71C8712A46D1E7D0010020C5
:1057D00080847E418084EE3F38B56C4620706170D5
:1057E000A270E37004226946952000F0C9F938BD23
:1057F0003EB5044600200090019002902449207894
:105800008978884201D000F04DF82078002814D023
:10581000012811D1A18906220B0A68460370417044
:10582000A17B8170E17BC170217C0171617C417140
:1058300069468C2000F0A4F93EBD607AF12802D0C0
:10584000F22808D00EE01348FFF734FF1248FFF7A4
:105850001FFF022006E01148FFF72CFF1048FFF75A
:1058600017FF0620618809220B0A69460B70A3788E
:105870004B7023798B706379CB70A3790B71E379CB
:105880004B71237A8B71C871A07A0872D0E700003F
:10589000D0010020FFFF0000058000000F1D000068
:1058A0002110000001B56846044900788870012283
:1058B00069468A2000F064F908BD0000D00100208C
:1058C0000A4610B50146002000F03CF910BD01B5B4
:1058D00001226946962000F053F908BD38B5104CF6
:1058E00005462078002804D12846FFF71BFD01203B
:1058F00020702846FAF744FE00220A4BFAF79EFD74
:10590000FAF74CFE020E69460A70020C4A70020A4F
:105910008A70C8700422862000F032F938BD000079
:10592000D00100208084EE3F10B5022100F098F8ED
:1059300010BD000008B5074A05215170020C6946E8
:105940000A70020A4A7088700322822000F018F957
:1059500008BD0000D001002038B5044609490520E3
:1059600048709621084800F028F9210C684601701B
:10597000210A4170847003226946822000F000F9F8
:1059800038BD0000D0010020AC0800001CB5030C9D
:105990006A461370030A53709070080CD070080A9E
:1059A0001071517106226946942000F0E9F802490D
:1059B000062048701CBD0000D001002001B5012266
:1059C0006946932000F0DCF808BD000001B5FFF740
:1059D000A6FC01226946842000F0D2F8014900208B
:1059E000487008BDD001002001B501226946802021
:1059F00000F0C6F8684601780348002902D0022169
:105A0000417008BD0121FBE7D001002001B5012252
:105A100069469F2000F0B4F808BD014610B51B2070
:105A20000822800100F0CFF8002010BD08B5074A19
:105A300004215170020C69460A70020A4A7088708B
:105A40000322832000F09CF808BD0000D001002054
:105A500010B500221146D12000F092F810BD0000D0
:105A6000F8B504460D460020FFF7C0FC02271B4E88
:105A7000FF43012809D00123002207210420FFF75A
:105A8000ABFE162C19DD16241AE00F2C09D00123C9
:105A90001A4600210420FFF79FFE0E2C08DB0E247F
:105AA00009E001231A4600210620FFF795FEF6E7DC
:105AB000BC4200DA3C46182103E0BC4200DA3C4616
:105AC0003821304600F079F86846047045700222AB
:105AD00069468E2000F054F8F8BD0000E708000089
:105AE00070B504460A488078002810D1D725ED000B
:105AF0002846FFF758FD4008E1054000C90F014363
:105B0000284600F05AF8E1B2681C00F056F870BD63
:105B1000D0010020024980200A699043FBD07047E1
:105B20000004004870B50125ED030924E406A562D0
:105B3000C02000F085FA002000F082FAA561FFF78E
:105B4000E9FF70BDF7B516460446FFF725FC0125B1
:105B5000ED030927FF06BD620E2000F071FA204612
:105B600000F06EFA002405E00198005D00F068FA8C
:105B7000641CA4B2B442F7D3BD61FFF7CBFFFEBDF6
:105B8000F7B51646FFF708FC0125ED030927FF06C8
:105B9000BD62009800F054FA002405E00198005D11
:105BA00000F04EFA641CA4B2B442F7D3BD61009871
:105BB000842801D0FFF7AEFFFEBD13B5012201A975
:105BC00000F001F81CBDF7B516460446FFF7E4FBEC
:105BD0000125ED030927FF06BD620D2000F030FA14
:105BE000200A00F02DFAE0B200F02AFA002405E0C5
:105BF0000198005D00F024FA641CA4B2B442F7D30B
:105C0000BD61FFF787FFFEBD10B5184C6168491CE8
:105C1000616017490180A18841801649CA6C828061
:105C2000496D8160112181831349C183A1684A01B3
:105C30001249511800228B5CFF2B03D02022FAF767
:105C4000BBFF05E0521C202AF5D3202200F0D2FC35
:105C5000A0682060401CA060400101218902203022
:105C6000884201D90020A060002010BD98000020CB
:105C7000AA55000040130020A55A000000C80008E3
:105C800010B514460A46012802D0022806D00DE0BD
:105C900021461046FEF740FE054804E02146104626
:105CA000FEF748FE0348816F491C8167204610BDFE
:105CB000E0020020740300200B0702881B0F012163
:105CC00099400A43028070470907090F01238B405E
:105CD0000188002A01D0194300E0994301807047F0
:105CE00010B5002A02D0FFF7E7FF10BDFFF7DAFA80
:105CF00010BD0907090F01238B400188002A01D03C
:105D0000194300E0994301807047000070B50B050E
:105D10001B0E204C5B000D071C192D0F030000F01B
:105D2000BAFC09060B14191E22272C313600FF2954
:105D30002DD89520800003E0FF2928D89D208000E1
:105D400020182946FFF7D5FF21E0FF291FD8A520FD
:105D50008000F5E780291AD2FD208000F0E7802935
:105D600015D20D48ECE7402911D2AD208000E7E7BD
:105D700040290CD2B5208000E2E7802907D20648EE
:105D80002030DDE7802902D203488030D8E70020A8
:105D900070BD0000C00D0020140400000121C903E3
:105DA000034A002801D0916270479161704700005A
:105DB0000008004801218903034A002801D09162AC
:105DC00070479161704700000008004801210922D6
:105DD000C902D206002801D09161704791627047D4
:105DE00001214903034A002801D091627047916163
:105DF0007047000000080048F0B5304C4B001C19FB
:105E00000923DB01E6180B23DB01E51892B28A288F
:105E10003DD00EDC294F4B00DF1909239B01FF18F1
:105E20008338030000F037FC0714181C21262D4688
:105E3000480099283ED006DC8B282CD08C2831D005
:105E40008D2839D133E0A12834D0FE2834D131E077
:105E5000102931DABA822FE010292DDABA862BE028
:105E6000102929DA0520C00108E0082924DA0F20CA
:105E7000800114E008291FDA0120800220188282A4
:105E80001AE0802918DAB28616E0AA8614E0802982
:105E900012DAB28210E040290EDA0D2080012018BB
:105EA000828609E0402907DA0B208001F7E74029C4
:105EB00002DAE8E78029E8DB0020F0BDC00D002011
:105EC000F0B591B0002600F0A7FEFBF733F807907D
:105ED0001021394800F000FF0A90FBF72BF80490DE
:105EE0001021354800F0A4FE0990FBF723F8039039
:105EF0001021314800F0B8FE0290FBF71BF8054670
:105F000010212D4800F0C8FE0190FBF713F82B4933
:105F100004468868012210438860901E0861284862
:105F20000861254B00201A5C0A70401C1028FADB1F
:105F30000F68FAF7FFFF029902970091214F08902E
:105F4000B81921A1099B0A9A00F07AFB86190898D2
:105F5000039A011B601B0291019004990398AA1AED
:105F6000431A084607990092421AB81920A100F076
:105F700067FB84190BA8FDF7E7F826484268012063
:105F8000000402403819134623A100F059FB0419FC
:105F9000381926A10B9A00F053FB01193846FEF779
:105FA000ADFC01210D20FDF727FA2449032088606C
:105FB000002011B0F0BD0000407300080030024026
:105FC00001A00000E00100200D0A435243202025DB
:105FD00030345820202530345820202530345820A3
:105FE00020253034582020253034580D0A00000078
:105FF00074696D6520253034642020253034642098
:10600000202530346420202530346420202530348D
:10601000640D0A00001002404D61696E536F757285
:106020006365202578202564200D0A007379736349
:106030006C6B202564200D0A000000000000002089
:1060400000220F4902E0521C322A03DC8B689B07B6
:10605000DB0FF8D00873002002E0401C322803DC7C
:106060008A681206D20FF8D1002002E0401C3228C4
:1060700003DC8A68D207D20FF8D0C868C0B2704774
:106080000030014030B50023174918464B604200EC
:106090005218401C1381FF28F9DD00220524134803
:1060A000E40155002D182D19521CAB82102AF8DB83
:1060B00000220924E40155002D182D19521CAB862D
:1060C000FF2AF8DD00221024D3001B1840331D8B5B
:1060D000521CA5431D83402AF6DB012008600449B9
:1060E0004882002030BD0000380B0020C00D002089
:1060F0007415002010B500220C48092302600C49D9
:1061000010469B0144006418E418401CA286102825
:10611000F8DB002001239B0244006418E418401CB3
:10612000A2820828F8DB002010BD0000380B0020F8
:10613000C00D002010B5402802DB0020C04310BD78
:106140000B4AC10089180B4640331C7EA4060DD5AE
:10615000400080180B220024920180188486054894
:1061600000684865188B202188431883002010BDE3
:10617000C00D0020DC01002010B5FAF7B3FFFBF7DB
:1061800055FB10BD70B594B030216846FAF726F87B
:10619000002501240E9520040990009405200F95F8
:1061A000C0040D95022601940A900C9508960B9454
:1061B0006846FBF733F9002803D0862115A000F0CC
:1061C0003DFA07200C900E9501210D960F950CA815
:1061D000FBF74CF8002803D092210EA000F02EFA15
:1061E000109410A81294FAF7CDFF002803D0A12133
:1061F00008A000F023FA4B208001FBF7FFFA0420EF
:10620000FBF7B6FA00221146501EFAF7B7FF14B09A
:1062100070BD00002E2E5C436F6D4C69625C537242
:10622000635C4253502E63001348016801221143FE
:1062300001604168114A114041600168104A1140F3
:1062400001600168012292049143016041683F228C
:10625000120491434160C16A09090901C162016BDD
:10626000FF22143291430163416B490849004163A5
:106270000021816070470000001002400CB8FF0848
:10628000FFFFF6FE04480169C907C90F02D00121CA
:10629000C9430161704700000010004070B51B4CFD
:1062A000E0698006C10F1A4811D01A4A0121116015
:1062B000194A11600169491C0161A18C4268521C94
:1062C0004260174B154D1A68A954521C1A60E169B7
:1062D0000907C90F04D008212162C169491CC161A5
:1062E0002068C006C00F07D0E069C006C00F03D009
:1062F0001020206200F03CF8E0694006C00F03D097
:106300004020206200F074F870BD000000380140A9
:10631000E002002044000020480000200804002083
:106320003C00002010B5104CE069E0690007C00F88
:1063300005D0082020620D48C169491CC161206850
:10634000C006C00F07D0E069C006C00F03D0102000
:10635000206200F09DF8E0694006C00F03D04020A5
:10636000206200F0E5F810BD0044004074030020F6
:106370000548416A491C416204490968002901DD58
:106380000121C16770470000E00200203C000020AE
:10639000F8B5144E0C46054602213046FCF7EAFDDE
:1063A00010200090104B2A4602213046FCF7CCFD0D
:1063B000224602213046FCF70FFE02213046FCF750
:1063C000E5FD0A4804630121417202213046FCF7D1
:1063D000E9FD054828388168802211438160204604
:1063E000F8BD00000000024028380140E002002013
:1063F0000248016A491C016270470000E002002067
:1064000010B50A48407A00280DD1084C206F583446
:10641000002808D12046FAF7DDFC0146E268206832
:106420008018FFF7B5FF002010BD0000E00200203B
:10643000F8B5144E0C46054605213046FCF79AFD8A
:10644000002000902B46104A05213046FCF77CFDC9
:10645000224605213046FCF7BFFD05213046FCF7FA
:1064600095FD0A4844630121817205213046FCF7FD
:1064700099FD05482438816840221143816000203D
:10648000F8BD0000000002402444004074030020D6
:106490000A480B4900794058802180B2091A0948FE
:1064A000012201600848C267426A521C4262002908
:1064B00003DD01200549000748607047507300085C
:1064C00004000240400000207403002000ED00E0C2
:1064D000F8B5144E0C46054604213046FCF74AFD3B
:1064E00010200090104B2A4604213046FCF72CFD6A
:1064F000224604213046FCF76FFD04213046FCF7AC
:1065000045FD0A4804630121417204213046FCF72D
:1065100049FD054828388168802211438160204662
:10652000F8BD000000000240284400407403002031
:106530000248016A491C0162704700007403002090
:106540000A4610B503494B885B1C4380FAF734FBBD
:10655000002010BD007C000870B50C460B494118A6
:10656000002B08D00A4D4519012B03D0094B9B8AFB
:10657000002B00D129468005204603D000F03AF8D0
:10658000002070BDFAF718FBFAE700000080000851
:1065900000A000087415002070B54188134A491CFA
:1065A0004180114901807E210A5280241049002235
:1065B000134663435D180023EE5CFF2E03D0521C8C
:1065C000082AF5DB0AE05B1CA342F5DB082A05D2AA
:1065D00062435118802200F00DF802E08022FAF7A1
:1065E000EBFA002070BD0000AA550000A55A00007B
:1065F00000C00008F7B515460E46FAF75BFD00240B
:10660000AF0808E00099A0000A5881190023022071
:10661000FAF712FD641CA742F4D87C006D0808E06C
:10662000009960000A5A811900230120FAF704FD3D
:10663000641CA542F4D8FAF7F5FCFEBDFEE70000A5
:106640000FB410B504A9074B02AA039800F040F854
:10665000044602A9002000F075FA204610BC08BCD0
:1066600004B01847456B00082021020C01D010210E
:106670001046020A01D010460839020901D010461E
:10668000091F820801D01046891E420801D0881EC9
:106690007047081A704730B47446641E2578641C2D
:1066A000AB4200D21D46635D5B00E31830BC184767
:1066B00002E008C8121F08C1002AFAD170477047CB
:1066C000002001E001C1121F002AFBD17047000029
:1066D000FFB591B00F460546002606E025280AD0F2
:1066E000149A139990476D1C761C28780028F5D1D0
:1066F000304615B0F0BD002400940121F34A029405
:1067000000E004436D1C2B780846203B9840104263
:10671000F7D128782A280ED0022128780246303A6C
:10672000092A15D8009A0A235A43303A80180C4394
:106730006D1C0090F1E701CF0090002805DA0120E0
:1067400040030443009840420090022004436D1C23
:1067500028782E2815D10420044368786D1C2A2837
:106760000AD101CF6D1C02900BE002990A2251431D
:10677000303940186D1C02902878014630390929BB
:10678000F3D928786C2810D006DC4C281AD0682859
:106790000ED06A2817D104E0742813D07A2812D1B9
:1067A00010E00120400504430CE00121090501E04F
:1067B000032109050C436978814203D101200005BA
:1067C00024186D1C6D1C287803906E281ED00CDCDC
:1067D000632831D004DC00288AD0582811D1B2E0D7
:1067E00064287BD069280CD178E073282DD004DC94
:1067F0006F2870D0702804D1A7E075286CD0782855
:106800006BD0149A13999047761C62E06002400F97
:10681000022807D003280AD0042838680AD0066066
:106820003F1D56E03868F11706604160F8E73868A8
:106830000680F5E70670F3E73878694608740020AB
:10684000487404A80390012003E0386803900020F6
:10685000C0433F1D61070FD5002101E00199491C8C
:10686000029A0191914213DA8142F7DB019A03996E
:10687000895C0029F2D10BE0002101E00199491C5B
:1068800001918142FADB019A0399895C0029F5D1D3
:1068900001990098139A401A00902146149B00F029
:1068A0003BF901998019461807E00398039900788D
:1068B000491C0391149A139990470198401E019026
:1068C000401CF2D12146149B139A009800F014F951
:1068D00086196D1C09E741E033E034E00A2000210D
:1068E000049005916002410F022905D001CFC21723
:1068F0009446032905D007E0FF1DFF08FF0003CFE2
:1069000006E000B2C2179446042902D140B2C11772
:106910008C4600226146944506DA0A460021404230
:1069200091418C462D2102E0210504D52B216A4698
:106930001176012103E0E10701D02021F7E7019161
:1069400054E00A200BE0102009E010200490002100
:106950000420044308200591029003E00820002150
:10696000059104906002410F022905D001CF002259
:106970009446032906D006E0FF1DFF08FF0003CF61
:106980008C4603E080B2042900D1C0B200210191FD
:1069900021072BD50399702906D0049A1021059B55
:1069A0004A401A4305D00EE040216A461176012183
:1069B00008E06146014306D030216A46117603990A
:1069C000517602210191049A0821059B4A401A43FD
:1069D0000CD16146014301D1610707D530216A46D8
:1069E0001176012101910299491E029103995829BA
:1069F00004D037A103910FA90F910DE039A1F9E758
:106A00006146059B049AF9F7FBFD039B8C469B5C52
:106A10000F9A521E0F92137061460143F0D10F98E6
:106A200007A9081A20300390600704D5012000044C
:106A30008443029801E0012002900399884201DD1D
:106A4000401A00E0002041180290019809180098AF
:106A5000401A0090E00306D42146149B139A009834
:106A600000F05AF886190020049008E006A9085C96
:106A7000149A139990470498401C761C049001992D
:106A80008842F3DBE0030CD52146149B139A00984F
:106A900000F042F8861904E0149A302013999047C8
:106AA000761C0299481E02900029F5DC08E00F9838
:106AB0000F990078491C0F91149A13999047761CEE
:106AC0000399481E03900029F1DCFBE60928010028
:106AD0003031323334353637383961626364656654
:106AE0000000000030313233343536373839414216
:106AF0004344454600000000F8B5044600251E4604
:106B00001746880404D405E039462020B0476D1CA0
:106B1000641EF9D52846F8BDFFB50446002581B0AE
:106B20001E46C80301D5302700E02027880404D57D
:106B300005E038460399B0476D1C641EF9D5284618
:106B400005B0F0BD0A68531C0B6010707047000060
:106B5000F8B54A002B4B520DD6182B4A0C46054669
:106B6000142E2BDA002E12DA284BF9F74DFB0022F7
:106B70001346F9F731FD40D2002C03DA0124E40773
:106B800000253AE02046284337D0214C14E0214F1D
:106B90000B46F7403B402B4331D01C4BF9F734FBFD
:106BA00000221346F9F718FD27D2002C03DD01203F
:106BB0000005F0400419BC4300251EE0332E1EDC06
:106BC00033460027143BFF43DF40384217D00F4BBA
:106BD000F9F7C4FB00221346F9F7FEFC0DD2002C96
:106BE0000ADD142E0CD03420811B0120884040196E
:106BF000A84200D2641C0546BD4321462846F8BD84
:106C0000641CF9E701FCFFFF9C7500883CE4377EBB
:106C10000000F03FFFFF0F0010B50A2101A0FDF7B3
:106C20006DFE10BD1B5B324A1B5B303B30480000E1
:106C300030B503460A4800290ED11A78094C504055
:106C40000022C50702D04008604000E04008521C06
:106C5000D2B2082AF5D35B1C491EEED230BD00002B
:106C6000FFFF000001A0000070B50A4DFF23EE1DDC
:106C70001A46F93605E0047854402A5D5A40335DDF
:106C8000401C0C46491E89B2002CF4D11802104356
:106C900070BD00005675000870B504460C4800220F
:106CA0000C4E11E02578521C2B4643401B07DB0E8F
:106CB000F35A00094340280958400007C00E305AD3
:106CC0001B09584092B2641C8A42EBD370BD00008D
:106CD000FFFF00005677000810B5084A084B07E090
:106CE000047854402406E40D1C5B120A6240401CE8
:106CF000491EF5D2D04380B210BD0000FFFF000056
:106D00005673000810B572B604220A498A614A0116
:106D1000131102248C62104201D08B6100E08B625F
:106D2000520802248C61002AF3D104208862886111
:106D300062B610BD00040048F8B54A002B4B520D56
:106D4000D6182B4A0C460546142E2BDA002E12DAE2
:106D5000284BF9F759FA00221346F9F73DFC40D2C7
:106D6000002C02DB002425463BE06000400828435D
:106D700037D0214C14E0214F0B46F7403B402B43CA
:106D800031D01C4BF9F740FA00221346F9F724FCE6
:106D900027D2002C03DA01200005F0400419BC437F
:106DA00000251EE0332E1EDC33460027143BFF4334
:106DB000DF40384217D00F4BF9F7D0FA00221346C4
:106DC000F9F70AFC0DD2002C0ADA142E0CD034206C
:106DD000811B012088404019A84200D2641C05464E
:106DE000BD4321462846F8BD641CF9E701FCFFFFBE
:106DF0009C7500883CE4377E0000F0BFFFFF0F0069
:106E000006C00021016041608160C1600122026111
:106E100041610846704700001CB5FF4D0127FF2067
:106E20002F830530FD4B80220090991AFC48FAF719
:106E300049FD4026FB4B3246991BFB480096FAF76A
:106E400041FDFAF757F90021F84B08460A4660243D
:106E50006243D21850609060106150619061D061BF
:106E6000106290625062D062491C10630929EDDB08
:106E7000EF4C00202067EF48C06A6066EE4800686B
:106E8000A066EE48406AE066FFF77CF9ED49EC4801
:106E90000860FAF727FDFCF727FBFCF711FBFBF76F
:106EA0000FFDE948FEF7D0F92F83FEF7C8F9A0637C
:106EB0006063E64801210170E54800210170E54862
:106EC00001210170E44801700846E4490870E1209E
:106ED000E34940020860FCF78DFCFCF71DFDFCF760
:106EE000A5FBE049486830434860FCF7FFFBFCF72E
:106EF00095FAFCF781FBFCF753FCDB4801680122A3
:106F000011430160D948026820210A4302600168E8
:106F10001022114301600168314301608021D4488F
:106F2000FFF786FAD3480168102211430160016817
:106F3000314301600A20FAF713F80120FEF750FFF1
:106F40000020FEF737FF0020FDF7A4FC0120F9F731
:106F50001DFEC948FFF7D6FE0120F9F721FE0020EB
:106F6000FEF734FFFEF7ACFFF9F7E4FF60660020A0
:106F700028826882B448C0882882288A01280AD1D9
:106F8000FAF75AFC208F202108406882688A00287E
:106F900001D0FFF777F8B94E5A207084A08E010710
:106FA0008006090FC00FFBF7F1FEFBF75DFF112113
:106FB000B3488901411800910F21C9014718B14D0B
:106FC0000020287001206870F9F7B4FF2861FAF7F3
:106FD00083F80190FEF733F905468F48008AC00711
:106FE0000BD0A806208F04D5800606D4FFF74AF8F8
:106FF00003E0800601D5FFF77DF8A5630198E06303
:107000000920C0060069B8849F480069F8849F4839
:10701000006938859E4800697885F9F713FF80B2CA
:10702000B082FFF76FFEF9F785FF964D68619948CA
:107030000068002801D00020B082206CC006C00E7D
:1070400002281CD1F9F70AFC9248016800290ED0E9
:107050000021B18290490A68002A10D100680860B6
:107060008E4800688E490860FDF77CF807E08A4981
:107070000A68002A03D000680860FDF78BF8894889
:10708000006E80470120FBF70DFE6348008A01284F
:107090000BD16148818A002927D08349A960C18A20
:1070A00082480160A868FDF77DF8606E69696166D5
:1070B000081AA066E16E884200D2E066216F88421D
:1070C00000D92067F9F736FFA861614800780028E9
:1070D00006D061480078002802D00220FAF73EFD71
:1070E0000198800403D5012002E07149D6E7002011
:1070F00028700198000501D5012000E0002068708B
:107100005448007800280ED06A480168890401D5E7
:10711000012100E0002129700068000501D501204F
:1071200000E000206870606C002801D0401E6064A0
:10713000A06C002801D0401EA0643748018B0029B4
:107140001FD06878FEF74CFE6878FEF733FE68784B
:10715000FEF724FE6878002801D1012000E000201D
:10716000FEF734FEF9F7E6FEE861A08EC00628D5EA
:107170005148818A0098C1864F49C08A4039888623
:1071800024E0008A01280FD0606C002810D06878B5
:10719000FEF726FEA06C00280CD06878FEF70AFEE9
:1071A0006878FEF7FBFDDAE7444800680028EFD076
:1071B0002878EDE70020FEF7FDFD0020FEF7EEFD4C
:1071C000CBE70098B18AC186C08AB086F9F7B2FED3
:1071D0002862B08EFDF75EFBF9F7ACFE0A2168620B
:1071E0000846F8F771FF0220401C4028FCDB206CA9
:1071F000401C206432480168002970DD084AD26FC3
:10720000002A6CD08AB22F490120FCF74DFC0028DF
:107210005ED02B482B4957E074150020141600202F
:10722000E0020020581700207403002028060020E8
:107230004013002080F7FF1F3000002000100240A4
:107240001027000014000020400D002050000020F6
:107250004C0000204D00002057000020510000206D
:107260003400002000300140001000400038014090
:107270008804002000440040FFFF000000100020B0
:10728000C00D0020C800002000040048000800488D
:10729000000C0048BC000020C00000201C000020A2
:1072A000C40000202C78000800A0000894000020F2
:1072B0000080000868000020C0110020380B00206A
:1072C0003C0000200804002002680120FAF75EFF5D
:1072D0001249002008601249C86713E0FFE711490E
:1072E000686888420DD9104841680122120511438F
:1072F00041604168520003235B059943114341609B
:1073000001E0401C686009480078002802D0002095
:10731000F9F726FE07490648086050E63C000020C1
:10732000E0020020C0270900003801404D00002085
:10733000AAAA00000030004010B5F9F713FA10BDFA
:10734000112233445566778899AABBCCDDEEFF0045
:10735000081C304458000000891112239B32244637
:10736000AD573665BF74488CC19D5AAFD3BE6CCA49
:10737000E5DB7EE9F7F88110080193331A22A55660
:107380002C47B7753E64C99C408DDBBF52AEEDDA29
:1073900064CBFFF976E802218B301002991326673F
:1073A000AF763444BD554AADC3BC588ED19F6EEB09
:1073B000E7FA7CC8F5D983310A2091121803A77720
:1073C0002E66B5543C45CBBD42ACD99E508FEFFBE9
:1073D00066EAFDD874C904428D5316619F7020047B
:1073E000A9153227BB364CCEC5DF5EEDD7FC6888C9
:1073F000E1997AABF3BA85520C4397711E60A114E0
:107400002805B3373A26CDDE44CFDFFD56ECE998A8
:107410006089FBBB72AA06638F7214409D512225BE
:10742000AB343006B9174EEFC7FE5CCCD5DD6AA988
:10743000E3B8788AF19B87730E6295501C41A3359F
:107440002A24B1163807CFFF46EEDDDC54CDEBB968
:1074500062A8F99A708B088481951AA793B62CC2FA
:10746000A5D33EE1B7F04008C919522BDB3A644E70
:10747000ED5F766DFF7C899400859BB712A6ADD237
:1074800024C3BFF136E0C1184809D33B5A2AE55E50
:107490006C4FF77D7E6C0AA583B4188691972EE316
:1074A000A7F23CC0B5D14229CB38500AD91B666F30
:1074B000EF7E744CFD5D8BB502A499961087AFF3F7
:1074C00026E2BDD034C1C3394A28D11A580BE77F10
:1074D0006E6EF55C7C4D0CC685D71EE597F4288052
:1074E000A1913AA3B3B2444ACD5B5669DF78600CF0
:1074F000E91D722FFB3E8DD604C79FF516E4A990B7
:107500002081BBB332A2C55A4C4BD7795E68E11CCF
:10751000680DF33F7A2E0EE787F61CC495D52AA195
:10752000A3B03882B193466BCF7A5448DD59622DAF
:10753000EB3C700EF91F8FF706E69DD414C5ABB176
:1075400022A0B9923083C77B4E6AD5585C49E33D8F
:107550006A2CF11E780F00C1814001C0804101C03A
:10756000804100C1814001C0804100C1814000C113
:10757000814001C0804101C0804100C1814000C103
:10758000814001C0804100C1814001C0804101C0F3
:10759000804100C1814001C0804100C1814000C1E3
:1075A000814001C0804100C1814001C0804101C0D3
:1075B000804100C1814000C1814001C0804101C0C3
:1075C000804100C1814001C0804100C1814000C1B3
:1075D000814001C0804101C0804100C1814000C1A3
:1075E000814001C0804100C1814001C0804101C093
:1075F000804100C1814000C1814001C0804101C083
:10760000804100C1814001C0804100C1814000C172
:10761000814001C0804100C1814001C0804101C062
:10762000804100C1814001C0804100C1814000C152
:10763000814001C0804101C0804100C1814000C142
:10764000814001C0804100C1814001C0804101C032
:10765000804100C1814000C0C101C30302C2C6060F
:1076600007C705C5C404CC0C0DCD0FCFCE0E0ACA7A
:10767000CB0BC90908C8D81819D91BDBDA1A1EDECA
:10768000DF1FDD1D1CDC14D4D515D71716D6D2127A
:1076900013D311D1D010F03031F133F3F23236F68A
:1076A000F737F53534F43CFCFD3DFF3F3EFEFA3A3A
:1076B0003BFB39F9F83828E8E929EB2B2AEAEE2ECA
:1076C0002FEF2DEDEC2CE42425E527E7E62622E23A
:1076D000E323E12120E0A06061A163A3A26266A68A
:1076E000A767A56564A46CACAD6DAF6F6EAEAA6AFA
:1076F0006BAB69A9A86878B8B979BB7B7ABABE7E4A
:107700007FBF7DBDBC7CB47475B577B7B67672B2F9
:10771000B373B17170B05090915193535292965689
:107720005797559594549C5C5D9D5F9F9E5E5A9AB9
:107730009B5B99595898884849894B8B8A4A4E8E49
:107740008F4F8D4D4C8C44848545874746868242B9
:10775000438341818040000001CC01D8001401F036
:10776000003C002801E401A0006C007801B4005046
:10777000019C01880044010F070100010001040180
:1077800010100000000000000000000006000000D3
:10779000AA550000000100000000000001000100E7
:1077A00000090000000000000000020000000009C5
:1077B00000000000000000000000000000000000C9
:1077C0000000000000000000101010101010101039
:1077D0001010101010101010100020003000400089
:1077E00050006000030000000400000005000000DD
:1077F000060000000700000008000000090000006B
:107800000A0000000B0000000C0000001100A55A47
:10781000AA55000000000000000000000000000069
:10782000081C304458081C3044580000414A0008E5
:107830001D4A0008D54C0008A14C0008854B0008E3
:10784000B54B00083D4D0008094F0008D549000818
:1078500069500008614C0008395000085950000870
:10786000014C00086150000825500008F94B000841
:10787000ED510008E94B0008F5510008F14B0008F4
:10788000A94C0008054D00083B4A0008894A000839
:10789000314C0008014F000804050600C01200002A
:1078A0001F000000A816000017000000841C000044
:1078B0000F000000E42500001E000000B42D0000B1
:1078C00016000000083900000E0000002C4C0000DB
:1078D0001D000000685B00001500000074720000CD
:1078E0000D000000589800001C00000034B7000094
:1078F00014000000E8E400000C00000078310100F2
:107900001B000000686E01001300000034CA010073
:107910000B000000286202001A00000040DB020099
:10792000120000003C9303000A000000C0C20400E3
:107930001900000060B305001100000038200700A6
:107940000900000020A10700000000000000000066
:1079500000000000010203040607080900000000FF
:10796000010203048479000800000020E001000007
:1079700004080008E4790008E0010020F81B00007A
:10798000C066000801103201031F102713C2010452
:107990001340420F293E113B010107012AA92F295B
:1079A0000C32971AFF01013512800A1C086C496ECF
:1079B00009165D4809FCA9F1D24D624040085A30D1
:1079C000085A20085A10081159084BF03F085AE08D
:1079D000085AD0080936385AC00809363893B03FDB
:0479E000531BB7007E
:04000005080000B53A
:00000001FF
